 Proclist

 Timestamp is 543873e1 (Sat Oct 11 04:03:45 2014)

 Preferred load address is 10000000

 Start         Length     Name                   Class
 0001:00000000 00000204H .idata$5                CODE
 0001:00000204 00000004H .CRT$XCA                CODE
 0001:00000208 00000004H .CRT$XCZ                CODE
 0001:0000020c 00000004H .CRT$XIA                CODE
 0001:00000210 0000000cH .CRT$XIC                CODE
 0001:0000021c 00000004H .CRT$XIZ                CODE
 0001:00000220 00000004H .CRT$XPA                CODE
 0001:00000224 00000004H .CRT$XPZ                CODE
 0001:00000228 00000004H .CRT$XTA                CODE
 0001:0000022c 00000004H .CRT$XTZ                CODE
 0001:00000230 00003b28H .rdata                  CODE
 0001:00003d58 000000dcH .rdata$r                CODE
 0001:00003e40 0000000cH .rdata$sxdata           CODE
 0001:00003e4c 00000004H .rtc$IAA                CODE
 0001:00003e50 00000004H .rtc$IZZ                CODE
 0001:00003e54 00000004H .rtc$TAA                CODE
 0001:00003e58 00000004H .rtc$TZZ                CODE
 0001:00003e60 000128d3H .text                   CODE
 0001:00016733 00000014H .text$yd                CODE
 0001:00016748 00000244H .xdata$x                CODE
 0001:0001698c 0000008cH .idata$2                CODE
 0001:00016a18 00000014H .idata$3                CODE
 0001:00016a2c 00000204H .idata$4                CODE
 0001:00016c30 000008deH .idata$6                CODE
 0001:00017510 00000192H .edata                  CODE
 0002:00000000 00001048H .data                   DATA
 0002:00001060 00025dfcH .bss                    DATA
 0003:00000000 00000058H .rsrc$01                DATA
 0003:00000060 00000378H .rsrc$02                DATA

  Address         Publics by Value              Rva+Base       Lib:Object

 0000:00000000       __except_list              00000000     <absolute>
 0000:00000003       ___safe_se_handler_count   00000003     <absolute>
 0000:00000000       ___ImageBase               10000000     <linker-defined>
 0001:00000000       __imp__DuplicateTokenEx@24 10001000     advapi32:ADVAPI32.dll
 0001:00000004       __imp__OpenProcessToken@12 10001004     advapi32:ADVAPI32.dll
 0001:00000008       __imp__LookupPrivilegeValueW@12 10001008     advapi32:ADVAPI32.dll
 0001:0000000c       __imp__AdjustTokenPrivileges@24 1000100c     advapi32:ADVAPI32.dll
 0001:00000010       __imp__OpenThreadToken@16  10001010     advapi32:ADVAPI32.dll
 0001:00000014       __imp__SetThreadToken@8    10001014     advapi32:ADVAPI32.dll
 0001:00000018       __imp__RegConnectRegistryW@12 10001018     advapi32:ADVAPI32.dll
 0001:0000001c       __imp__RegQueryValueExW@24 1000101c     advapi32:ADVAPI32.dll
 0001:00000020       __imp__RegCloseKey@4       10001020     advapi32:ADVAPI32.dll
 0001:00000024       __imp__RegOpenKeyExW@20    10001024     advapi32:ADVAPI32.dll
 0001:00000028       __imp__GetUserNameW@8      10001028     advapi32:ADVAPI32.dll
 0001:0000002c       \177ADVAPI32_NULL_THUNK_DATA 1000102c     advapi32:ADVAPI32.dll
 0001:00000030       __imp__SetLastError@4      10001030     kernel32:KERNEL32.dll
 0001:00000034       __imp__VirtualFree@12      10001034     kernel32:KERNEL32.dll
 0001:00000038       __imp__VirtualAlloc@16     10001038     kernel32:KERNEL32.dll
 0001:0000003c       __imp__SetEvent@4          1000103c     kernel32:KERNEL32.dll
 0001:00000040       __imp__lstrcatW@8          10001040     kernel32:KERNEL32.dll
 0001:00000044       __imp__lstrcpyW@8          10001044     kernel32:KERNEL32.dll
 0001:00000048       __imp__FileTimeToSystemTime@8 10001048     kernel32:KERNEL32.dll
 0001:0000004c       __imp__lstrcmpiW@8         1000104c     kernel32:KERNEL32.dll
 0001:00000050       __imp__GetCurrentThreadId@0 10001050     kernel32:KERNEL32.dll
 0001:00000054       __imp__GetTickCount@0      10001054     kernel32:KERNEL32.dll
 0001:00000058       __imp__SystemTimeToTzSpecificLocalTime@12 10001058     kernel32:KERNEL32.dll
 0001:0000005c       __imp__GetLocalTime@4      1000105c     kernel32:KERNEL32.dll
 0001:00000060       __imp__GetSystemTimeAsFileTime@4 10001060     kernel32:KERNEL32.dll
 0001:00000064       __imp__CreateFileW@28      10001064     kernel32:KERNEL32.dll
 0001:00000068       __imp__SetPriorityClass@8  10001068     kernel32:KERNEL32.dll
 0001:0000006c       __imp__GetPriorityClass@4  1000106c     kernel32:KERNEL32.dll
 0001:00000070       __imp__lstrcmpW@8          10001070     kernel32:KERNEL32.dll
 0001:00000074       __imp__ResetEvent@4        10001074     kernel32:KERNEL32.dll
 0001:00000078       __imp__GetProcessTimes@20  10001078     kernel32:KERNEL32.dll
 0001:0000007c       __imp__WaitForMultipleObjects@16 1000107c     kernel32:KERNEL32.dll
 0001:00000080       __imp__CreateEventW@16     10001080     kernel32:KERNEL32.dll
 0001:00000084       __imp__CreateMutexW@12     10001084     kernel32:KERNEL32.dll
 0001:00000088       __imp__ReadProcessMemory@20 10001088     kernel32:KERNEL32.dll
 0001:0000008c       __imp__GetLastError@0      1000108c     kernel32:KERNEL32.dll
 0001:00000090       __imp__GetCurrentProcessId@0 10001090     kernel32:KERNEL32.dll
 0001:00000094       __imp__OpenProcess@12      10001094     kernel32:KERNEL32.dll
 0001:00000098       __imp__TerminateProcess@8  10001098     kernel32:KERNEL32.dll
 0001:0000009c       __imp__GetDateFormatW@24   1000109c     kernel32:KERNEL32.dll
 0001:000000a0       __imp__GetTimeFormatW@24   100010a0     kernel32:KERNEL32.dll
 0001:000000a4       __imp__FileTimeToLocalFileTime@8 100010a4     kernel32:KERNEL32.dll
 0001:000000a8       __imp__LocalFree@4         100010a8     kernel32:KERNEL32.dll
 0001:000000ac       __imp__FormatMessageW@28   100010ac     kernel32:KERNEL32.dll
 0001:000000b0       __imp__GetModuleHandleW@4  100010b0     kernel32:KERNEL32.dll
 0001:000000b4       __imp__GetProcAddress@8    100010b4     kernel32:KERNEL32.dll
 0001:000000b8       __imp__HeapReAlloc@16      100010b8     kernel32:KERNEL32.dll
 0001:000000bc       __imp__HeapSize@12         100010bc     kernel32:KERNEL32.dll
 0001:000000c0       __imp__LoadLibraryW@4      100010c0     kernel32:KERNEL32.dll
 0001:000000c4       __imp__EnterCriticalSection@4 100010c4     kernel32:KERNEL32.dll
 0001:000000c8       __imp__GetCurrentProcess@0 100010c8     kernel32:KERNEL32.dll
 0001:000000cc       __imp__DuplicateHandle@28  100010cc     kernel32:KERNEL32.dll
 0001:000000d0       __imp__lstrlenW@4          100010d0     kernel32:KERNEL32.dll
 0001:000000d4       __imp__lstrcpynW@12        100010d4     kernel32:KERNEL32.dll
 0001:000000d8       __imp__CreateThread@24     100010d8     kernel32:KERNEL32.dll
 0001:000000dc       __imp__TerminateThread@8   100010dc     kernel32:KERNEL32.dll
 0001:000000e0       __imp__CloseHandle@4       100010e0     kernel32:KERNEL32.dll
 0001:000000e4       __imp__Sleep@4             100010e4     kernel32:KERNEL32.dll
 0001:000000e8       __imp__ReleaseMutex@4      100010e8     kernel32:KERNEL32.dll
 0001:000000ec       __imp__WriteFile@20        100010ec     kernel32:KERNEL32.dll
 0001:000000f0       __imp__WaitForSingleObject@8 100010f0     kernel32:KERNEL32.dll
 0001:000000f4       __imp__GetCurrentThread@0  100010f4     kernel32:KERNEL32.dll
 0001:000000f8       __imp__LeaveCriticalSection@4 100010f8     kernel32:KERNEL32.dll
 0001:000000fc       __imp__MultiByteToWideChar@24 100010fc     kernel32:KERNEL32.dll
 0001:00000100       __imp__LCMapStringW@24     10001100     kernel32:KERNEL32.dll
 0001:00000104       __imp__QueryPerformanceCounter@4 10001104     kernel32:KERNEL32.dll
 0001:00000108       __imp__GetEnvironmentStringsW@0 10001108     kernel32:KERNEL32.dll
 0001:0000010c       __imp__WideCharToMultiByte@32 1000110c     kernel32:KERNEL32.dll
 0001:00000110       __imp__FreeEnvironmentStringsW@4 10001110     kernel32:KERNEL32.dll
 0001:00000114       __imp__GetModuleFileNameA@12 10001114     kernel32:KERNEL32.dll
 0001:00000118       __imp__DeleteCriticalSection@4 10001118     kernel32:KERNEL32.dll
 0001:0000011c       __imp__GetStartupInfoW@4   1000111c     kernel32:KERNEL32.dll
 0001:00000120       __imp__GetFileType@4       10001120     kernel32:KERNEL32.dll
 0001:00000124       __imp__InitializeCriticalSectionAndSpinCount@8 10001124     kernel32:KERNEL32.dll
 0001:00000128       __imp__SetHandleCount@4    10001128     kernel32:KERNEL32.dll
 0001:0000012c       __imp__GetStringTypeW@16   1000112c     kernel32:KERNEL32.dll
 0001:00000130       __imp__RaiseException@16   10001130     kernel32:KERNEL32.dll
 0001:00000134       __imp__HeapFree@12         10001134     kernel32:KERNEL32.dll
 0001:00000138       __imp__HeapAlloc@12        10001138     kernel32:KERNEL32.dll
 0001:0000013c       __imp__GetCommandLineA@0   1000113c     kernel32:KERNEL32.dll
 0001:00000140       __imp__GetCPInfo@8         10001140     kernel32:KERNEL32.dll
 0001:00000144       __imp__InterlockedIncrement@4 10001144     kernel32:KERNEL32.dll
 0001:00000148       __imp__InterlockedDecrement@4 10001148     kernel32:KERNEL32.dll
 0001:0000014c       __imp__GetACP@0            1000114c     kernel32:KERNEL32.dll
 0001:00000150       __imp__GetOEMCP@0          10001150     kernel32:KERNEL32.dll
 0001:00000154       __imp__IsValidCodePage@4   10001154     kernel32:KERNEL32.dll
 0001:00000158       __imp__TlsAlloc@0          10001158     kernel32:KERNEL32.dll
 0001:0000015c       __imp__TlsGetValue@4       1000115c     kernel32:KERNEL32.dll
 0001:00000160       __imp__TlsSetValue@8       10001160     kernel32:KERNEL32.dll
 0001:00000164       __imp__TlsFree@4           10001164     kernel32:KERNEL32.dll
 0001:00000168       __imp__UnhandledExceptionFilter@4 10001168     kernel32:KERNEL32.dll
 0001:0000016c       __imp__SetUnhandledExceptionFilter@4 1000116c     kernel32:KERNEL32.dll
 0001:00000170       __imp__IsDebuggerPresent@0 10001170     kernel32:KERNEL32.dll
 0001:00000174       __imp__HeapCreate@12       10001174     kernel32:KERNEL32.dll
 0001:00000178       __imp__HeapDestroy@4       10001178     kernel32:KERNEL32.dll
 0001:0000017c       __imp__ExitProcess@4       1000117c     kernel32:KERNEL32.dll
 0001:00000180       __imp__GetStdHandle@4      10001180     kernel32:KERNEL32.dll
 0001:00000184       __imp__GetModuleFileNameW@12 10001184     kernel32:KERNEL32.dll
 0001:00000188       __imp__IsProcessorFeaturePresent@4 10001188     kernel32:KERNEL32.dll
 0001:0000018c       __imp__RtlUnwind@16        1000118c     kernel32:KERNEL32.dll
 0001:00000190       \177KERNEL32_NULL_THUNK_DATA 10001190     kernel32:KERNEL32.dll
 0001:00000194       __imp__WNetAddConnection2W@16 10001194     mpr:MPR.dll
 0001:00000198       __imp__WNetCancelConnection2W@12 10001198     mpr:MPR.dll
 0001:0000019c       \177MPR_NULL_THUNK_DATA    1000119c     mpr:MPR.dll
 0001:000001a0       __imp__SysAllocString@4    100011a0     oleaut32:OLEAUT32.dll
 0001:000001a4       __imp__SysFreeString@4     100011a4     oleaut32:OLEAUT32.dll
 0001:000001a8       __imp__VariantClear@4      100011a8     oleaut32:OLEAUT32.dll
 0001:000001ac       \177OLEAUT32_NULL_THUNK_DATA 100011ac     oleaut32:OLEAUT32.dll
 0001:000001b0       __imp__GetWindowPlacement@8 100011b0     user32:USER32.dll
 0001:000001b4       __imp__GetParent@4         100011b4     user32:USER32.dll
 0001:000001b8       __imp__GetWindowThreadProcessId@8 100011b8     user32:USER32.dll
 0001:000001bc       __imp__wsprintfW           100011bc     user32:USER32.dll
 0001:000001c0       __imp__GetWindowLongW@8    100011c0     user32:USER32.dll
 0001:000001c4       __imp__IsIconic@4          100011c4     user32:USER32.dll
 0001:000001c8       __imp__GetWindowTextW@12   100011c8     user32:USER32.dll
 0001:000001cc       __imp__SystemParametersInfoW@16 100011cc     user32:USER32.dll
 0001:000001d0       __imp__SetForegroundWindow@4 100011d0     user32:USER32.dll
 0001:000001d4       __imp__EnumWindows@8       100011d4     user32:USER32.dll
 0001:000001d8       __imp__ShowWindowAsync@8   100011d8     user32:USER32.dll
 0001:000001dc       __imp__IsWindowVisible@4   100011dc     user32:USER32.dll
 0001:000001e0       \177USER32_NULL_THUNK_DATA 100011e0     user32:USER32.dll
 0001:000001e4       __imp__GetFileVersionInfoSizeW@8 100011e4     version:VERSION.dll
 0001:000001e8       __imp__GetFileVersionInfoW@16 100011e8     version:VERSION.dll
 0001:000001ec       __imp__VerQueryValueW@16   100011ec     version:VERSION.dll
 0001:000001f0       \177VERSION_NULL_THUNK_DATA 100011f0     version:VERSION.dll
 0001:000001f4       __imp__CoCreateInstance@20 100011f4     ole32:ole32.dll
 0001:000001f8       __imp__CoUninitialize@0    100011f8     ole32:ole32.dll
 0001:000001fc       __imp__CoInitialize@4      100011fc     ole32:ole32.dll
 0001:00000200       \177ole32_NULL_THUNK_DATA  10001200     ole32:ole32.dll
 0001:00000204       ___xc_a                    10001204     LIBCMT:crt0init.obj
 0001:00000208       ___xc_z                    10001208     LIBCMT:crt0init.obj
 0001:0000020c       ___xi_a                    1000120c     LIBCMT:crt0init.obj
 0001:0000021c       ___xi_z                    1000121c     LIBCMT:crt0init.obj
 0001:00000220       ___xp_a                    10001220     LIBCMT:crt0init.obj
 0001:00000224       ___xp_z                    10001224     LIBCMT:crt0init.obj
 0001:00000228       ___xt_a                    10001228     LIBCMT:crt0init.obj
 0001:0000022c       ___xt_z                    1000122c     LIBCMT:crt0init.obj
 0001:00000230       ??_C@_1BA@KLFBJALL@?$AAW?$AAm?$AAi?$AAG?$AAu?$AAi?$AAd?$AA?$AA@ 10001230     handles.obj
 0001:00000240       ??_C@_19DDLLJDOO@?$AAF?$AAi?$AAl?$AAe?$AA?$AA@ 10001240     handles.obj
 0001:0000024c       ??_C@_1BK@HCMNLOAL@?$AAI?$AAo?$AAC?$AAo?$AAm?$AAp?$AAl?$AAe?$AAt?$AAi?$AAo?$AAn?$AA?$AA@ 1000124c     handles.obj
 0001:00000268       ??_C@_17EKANHMLE@?$AAJ?$AAo?$AAb?$AA?$AA@ 10001268     handles.obj
 0001:00000270       ??_C@_1BK@GACLFIOK@?$AAW?$AAa?$AAi?$AAt?$AAa?$AAb?$AAl?$AAe?$AAP?$AAo?$AAr?$AAt?$AA?$AA@ 10001270     handles.obj
 0001:0000028c       ??_C@_19OBNDINH@?$AAP?$AAo?$AAr?$AAt?$AA?$AA@ 1000128c     handles.obj
 0001:00000298       ??_C@_17KACEIPNC@?$AAK?$AAe?$AAy?$AA?$AA@ 10001298     handles.obj
 0001:000002a0       ??_C@_1BA@LHDKDEEN@?$AAS?$AAe?$AAc?$AAt?$AAi?$AAo?$AAn?$AA?$AA@ 100012a0     handles.obj
 0001:000002b0       ??_C@_1BA@CBCBMBGJ@?$AAD?$AAe?$AAs?$AAk?$AAt?$AAo?$AAp?$AA?$AA@ 100012b0     handles.obj
 0001:000002c0       ??_C@_1BM@JIPCCEDL@?$AAW?$AAi?$AAn?$AAd?$AAo?$AAw?$AAS?$AAt?$AAa?$AAt?$AAi?$AAo?$AAn?$AA?$AA@ 100012c0     handles.obj
 0001:000002dc       ??_C@_1BA@OKEJPPOI@?$AAP?$AAr?$AAo?$AAf?$AAi?$AAl?$AAe?$AA?$AA@ 100012dc     handles.obj
 0001:000002ec       ??_C@_1M@EEEEDEMN@?$AAT?$AAi?$AAm?$AAe?$AAr?$AA?$AA@ 100012ec     handles.obj
 0001:000002f8       ??_C@_1BE@NPGPGCB@?$AAS?$AAe?$AAm?$AAa?$AAp?$AAh?$AAo?$AAr?$AAe?$AA?$AA@ 100012f8     handles.obj
 0001:0000030c       ??_C@_1O@FBKOCLFA@?$AAM?$AAu?$AAt?$AAa?$AAn?$AAt?$AA?$AA@ 1000130c     handles.obj
 0001:0000031c       ??_C@_1BE@EBMGBMON@?$AAE?$AAv?$AAe?$AAn?$AAt?$AAP?$AAa?$AAi?$AAr?$AA?$AA@ 1000131c     handles.obj
 0001:00000330       ??_C@_1M@JJBFPLJB@?$AAE?$AAv?$AAe?$AAn?$AAt?$AA?$AA@ 10001330     handles.obj
 0001:0000033c       ??_C@_1O@CDOGJPJJ@?$AAT?$AAh?$AAr?$AAe?$AAa?$AAd?$AA?$AA@ 1000133c     handles.obj
 0001:0000034c       ??_C@_1BA@NMDNJJOO@?$AAP?$AAr?$AAo?$AAc?$AAe?$AAs?$AAs?$AA?$AA@ 1000134c     handles.obj
 0001:0000035c       ??_C@_1M@JFPKKFCK@?$AAT?$AAo?$AAk?$AAe?$AAn?$AA?$AA@ 1000135c     handles.obj
 0001:00000368       ??_C@_1BK@KDPOKCA@?$AAS?$AAy?$AAm?$AAb?$AAo?$AAl?$AAi?$AAc?$AAL?$AAi?$AAn?$AAk?$AA?$AA@ 10001368     handles.obj
 0001:00000384       ??_C@_1BE@DNDHOCGP@?$AAD?$AAi?$AAr?$AAe?$AAc?$AAt?$AAo?$AAr?$AAy?$AA?$AA@ 10001384     handles.obj
 0001:00000398       ??_C@_11LOCGONAA@?$AA?$AA@ 10001398     handles.obj
 0001:000003fc       ??_C@_17CNPHIMPH@?$AA?$CF?$AAl?$AAs?$AA?$AA@ 100013fc     handles.obj
 0001:00000404       ??_C@_1BA@FDFONNEJ@?$AA?$CF?$AAs?$AA?5?$AA?$CI?$AA?$CF?$AAd?$AA?$CJ?$AA?$AA@ 10001404     handles.obj
 0001:00000414       ??_C@_1BE@ELICABCK@?$AA?$DM?$AAu?$AAn?$AAk?$AAn?$AAo?$AAw?$AAn?$AA?$DO?$AA?$AA@ 10001414     handles.obj
 0001:00000428       ??_C@_1BA@LGCEDAAB@?$AAT?$AAI?$AAD?$AA?3?$AA?5?$AA?$CF?$AAd?$AA?$AA@ 10001428     handles.obj
 0001:00000438       ??_C@_15GANGMFKL@?$AA?$CF?$AAs?$AA?$AA@ 10001438     handles.obj
 0001:00000440       ??_C@_19PEALEEJB@?$AAH?$AAK?$AAL?$AAM?$AA?$AA@ 10001440     handles.obj
 0001:0000044c       ??_C@_1BA@INBMCOAP@?$AAM?$AAA?$AAC?$AAH?$AAI?$AAN?$AAE?$AA?$AA@ 1000144c     handles.obj
 0001:0000045c       ??_C@_19NCHLBIN@?$AAH?$AAK?$AAC?$AAR?$AA?$AA@ 1000145c     handles.obj
 0001:00000468       ??_C@_1DC@OIDKFHBF@?$AAM?$AAA?$AAC?$AAH?$AAI?$AAN?$AAE?$AA?2?$AAS?$AAO?$AAF?$AAT?$AAW?$AAA?$AAR?$AAE?$AA?2?$AAC?$AAL?$AAA?$AAS?$AAS?$AAE?$AAS?$AA?$AA@ 10001468     handles.obj
 0001:0000049c       ??_C@_17PJOJPMPB@?$AAH?$AAK?$AAU?$AA?$AA@ 1000149c     handles.obj
 0001:000004a4       ??_C@_1BK@OEABCBLA@?$AAH?$AAK?$AAC?$AAU?$AA?2?$AAC?$AAl?$AAa?$AAs?$AAs?$AAe?$AAs?$AA?$AA@ 100014a4     handles.obj
 0001:000004c0       ??_C@_19JAPAIJDE@?$AAH?$AAK?$AAC?$AAU?$AA?$AA@ 100014c0     handles.obj
 0001:000004cc       ??_C@_1BC@PGMOPNLK@?$AA_?$AAC?$AAl?$AAa?$AAs?$AAs?$AAe?$AAs?$AA?$AA@ 100014cc     handles.obj
 0001:000004e0       ??_C@_19KGHAHCFG@?$AAU?$AAS?$AAE?$AAR?$AA?$AA@ 100014e0     handles.obj
 0001:000004ec       ??_C@_1BG@OKCBELMP@?$AA?2?$AAR?$AAE?$AAG?$AAI?$AAS?$AAT?$AAR?$AAY?$AA?2?$AA?$AA@ 100014ec     handles.obj
 0001:00000504       ??_C@_1O@EAOKCHFC@?$AA?$CF?$AA?9?$AA1?$AA3?$AAs?$AA?5?$AA?$AA@ 10001504     handles.obj
 0001:00000514       ??_C@_19DEJHOMFE@?$AA?9?$AA?$CF?$AAl?$AAu?$AA?$AA@ 10001514     handles.obj
 0001:00000520       ??_C@_1EC@MPDKEHCN@?$AA0?$AAx?$AA?$CF?$AA0?$AA2?$AAh?$AAx?$AA?$CF?$AA0?$AA2?$AAh?$AAx?$AA?$CF?$AA0?$AA2?$AAh?$AAx?$AA?$CF?$AA0?$AA2?$AAh?$AAx?$AA?$CF?$AA0?$AA2?$AAh?$AAx?$AA?$CF?$AA0?$AA2?$AAh?$AAx@ 10001520     handles.obj
 0001:00000564       ??_C@_17IJMNDCL@?$AA?$CF?$AAl?$AAu?$AA?$AA@ 10001564     handles.obj
 0001:0000056c       ??_C@_1BA@IGEMANKH@?$AA?2?$AAS?$AA?9?$AA?$CF?$AAl?$AAu?$AA?9?$AA?$AA@ 1000156c     handles.obj
 0001:0000057c       ??_C@_1BG@OCPCMCEA@?$AA?$CF?$AA5?$AAX?$AA?5?$AA?5?$AA?$CF?$AA0?$AA8?$AAX?$AA?5?$AA?$AA@ 1000157c     handles.obj
 0001:00000594       ??_C@_1O@HAOIKAHJ@?$AA?$CF?$AAs?$AA?6?$AA?$CF?$AAs?$AA?6?$AA?$AA@ 10001594     handles.obj
 0001:000005a4       ??_C@_1CK@CLFOOHFA@?$AAE?$AAx?$AAp?$AAo?$AAr?$AAt?$AAH?$AAa?$AAn?$AAd?$AAl?$AAe?$AAs?$AAU?$AAn?$AAn?$AAa?$AAm?$AAe?$AAd?$AA?$AA@ 100015a4     PCFG.OBJ
 0001:000005d0       ??_C@_1BM@KMCHODLM@?$AAE?$AAx?$AAp?$AAo?$AAr?$AAt?$AAH?$AAa?$AAn?$AAd?$AAl?$AAe?$AAs?$AA?$AA@ 100015d0     PCFG.OBJ
 0001:000005ec       ??_C@_1CE@GNMOKOAL@?$AAE?$AAx?$AAp?$AAo?$AAr?$AAt?$AAP?$AAe?$AAr?$AAf?$AAo?$AAr?$AAm?$AAa?$AAn?$AAc?$AAe?$AA?$AA@ 100015ec     PCFG.OBJ
 0001:00000610       ??_C@_1CI@OFLGHPDG@?$AAE?$AAx?$AAp?$AAo?$AAr?$AAt?$AAM?$AAo?$AAd?$AAu?$AAl?$AAe?$AAV?$AAe?$AAr?$AAs?$AAi?$AAo?$AAn?$AA?$AA@ 10001610     PCFG.OBJ
 0001:00000638       ??_C@_1CC@OABICAMP@?$AAE?$AAx?$AAp?$AAo?$AAr?$AAt?$AAM?$AAo?$AAd?$AAu?$AAl?$AAe?$AAI?$AAn?$AAf?$AAo?$AA?$AA@ 10001638     PCFG.OBJ
 0001:0000065c       ??_C@_1CE@JIPJNDMD@?$AAE?$AAx?$AAp?$AAo?$AAr?$AAt?$AAE?$AAn?$AAv?$AAi?$AAr?$AAo?$AAn?$AAm?$AAe?$AAn?$AAt?$AA?$AA@ 1000165c     PCFG.OBJ
 0001:00000680       ??_C@_1CC@PNNAOHJC@?$AAA?$AAd?$AAd?$AAT?$AAo?$AAP?$AAl?$AAu?$AAg?$AAi?$AAn?$AAs?$AAM?$AAe?$AAn?$AAu?$AA?$AA@ 10001680     PCFG.OBJ
 0001:000006a4       ??_C@_1BO@NGDOFANC@?$AAA?$AAd?$AAd?$AAT?$AAo?$AAD?$AAi?$AAs?$AAk?$AAs?$AAM?$AAe?$AAn?$AAu?$AA?$AA@ 100016a4     PCFG.OBJ
 0001:000006c4       ??_C@_1BE@PKILIDFH@?$AAE?$AAn?$AAa?$AAb?$AAl?$AAe?$AAW?$AAM?$AAI?$AA?$AA@ 100016c4     PCFG.OBJ
 0001:000006d8       ??_7?$DialogBuilderBase@UFarDialogItem@@@@6B@ 100016d8     PCFG.OBJ
 0001:000006fc       ??_7PluginDialogBuilder@@6B@ 100016fc     PCFG.OBJ
 0001:00000720       ??_7?$DialogItemBinding@UFarDialogItem@@@@6B@ 10001720     PCFG.OBJ
 0001:00000728       ??_7PluginCheckBoxBinding@@6B@ 10001728     PCFG.OBJ
 0001:00000730       ??_7PluginRadioButtonBinding@@6B@ 10001730     PCFG.OBJ
 0001:00000738       ??_C@_15EFLNJKHH@?$AA?$CF?$AAu?$AA?$AA@ 10001738     PCFG.OBJ
 0001:00000740       ??_7PluginIntEditFieldBinding@@6B@ 10001740     PCFG.OBJ
 0001:00000748       ??_7PluginUIntEditFieldBinding@@6B@ 10001748     PCFG.OBJ
 0001:00000750       ??_C@_1O@BJPKKLLM@?$AAC?$AAo?$AAn?$AAf?$AAi?$AAg?$AA?$AA@ 10001750     PCFG.OBJ
 0001:00000760       ??_C@_13LHMFKAAD@?$AAM?$AA?$AA@ 10001760     Pclass.obj
 0001:00000764       ??_C@_13JCKOPPNP@?$AAK?$AA?$AA@ 10001764     Pclass.obj
 0001:00000768       ??_C@_1CC@EBBNDNOD@?$AAF?$AAu?$AAl?$AAl?$AAS?$AAc?$AAr?$AAe?$AAe?$AAn?$AAR?$AAe?$AAm?$AAo?$AAt?$AAe?$AA?$AA@ 10001768     Pclass.obj
 0001:0000078c       ??_C@_1CA@HLBJOHGN@?$AAF?$AAu?$AAl?$AAl?$AAS?$AAc?$AAr?$AAe?$AAe?$AAn?$AAL?$AAo?$AAc?$AAa?$AAl?$AA?$AA@ 1000178c     Pclass.obj
 0001:000007ac       ??_C@_1BK@DDBMMJCN@?$AAW?$AAi?$AAd?$AAt?$AAh?$AAs?$AAR?$AAe?$AAm?$AAo?$AAt?$AAe?$AA?$AA@ 100017ac     Pclass.obj
 0001:000007c8       ??_C@_1BI@FOOHDOCI@?$AAW?$AAi?$AAd?$AAt?$AAh?$AAs?$AAL?$AAo?$AAc?$AAa?$AAl?$AA?$AA@ 100017c8     Pclass.obj
 0001:000007e0       ??_C@_1BM@EDHFKJEJ@?$AAC?$AAo?$AAl?$AAu?$AAm?$AAn?$AAs?$AAR?$AAe?$AAm?$AAo?$AAt?$AAe?$AA?$AA@ 100017e0     Pclass.obj
 0001:000007fc       ??_C@_1BK@HMOODHKK@?$AAC?$AAo?$AAl?$AAu?$AAm?$AAn?$AAs?$AAL?$AAo?$AAc?$AAa?$AAl?$AA?$AA@ 100017fc     Pclass.obj
 0001:00000818       ??_C@_1O@CBODAMOP@?$AAM?$AAo?$AAd?$AAe?$AA?$CF?$AAd?$AA?$AA@ 10001818     Pclass.obj
 0001:00000828       ??_C@_15LNKNCLHH@?$AAS?$AAs?$AA?$AA@ 10001828     Pclass.obj
 0001:00000830       ??_C@_13DEFPDAGF@?$AA?0?$AA?$AA@ 10001830     Pclass.obj
 0001:00000834       ??_C@_19MPDKCIDK@?$AA?5?$AA?$CF?$AAs?$AA?5?$AA?$AA@ 10001834     Pclass.obj
 0001:00000840       ??_C@_1BA@MFHNOFIJ@?$AA?$CF?$AAs?$AA?3?$AA?5?$AA?$CF?$AAs?$AA?5?$AA?$AA@ 10001840     Pclass.obj
 0001:00000850       ??_C@_13HOIJIPNN@?$AA?5?$AA?$AA@ 10001850     Pclass.obj
 0001:00000854       ??_C@_17JJIMNMHK@?$AA?5?$AA?$CG?$AA?$FO?$AA?$AA@ 10001854     Pclass.obj
 0001:0000085c       ??_C@_1M@EJMLOAMM@?$AA?$CF?$AA?9?$AA2?$AA2?$AAs?$AA?$AA@ 1000185c     Pclass.obj
 0001:00000868       ??_C@_17DJGLCLAO@?$AA?$CF?$AAs?$AA?3?$AA?$AA@ 10001868     Pclass.obj
 0001:00000870       ??_C@_17JLFEDMMI@?$AA?$DP?$AA?$DP?$AA?$DP?$AA?$AA@ 10001870     Pclass.obj
 0001:00000878       ??_C@_1BO@EHJBCONC@?$AA?$CF?$AA0?$AA2?$AAd?$AA?3?$AA?$CF?$AA0?$AA2?$AAd?$AA?3?$AA?$CF?$AA0?$AA2?$AAd?$AA?$AA@ 10001878     Pclass.obj
 0001:00000898       ??_C@_1CE@OMPPCAIJ@?$AA?$CF?$AAd?$AA?5?$AA?$CF?$AA0?$AA2?$AAd?$AA?3?$AA?$CF?$AA0?$AA2?$AAd?$AA?3?$AA?$CF?$AA0?$AA2?$AAd?$AA?$AA@ 10001898     Pclass.obj
 0001:000008ec       ??_C@_1CO@PDLCNLLF@?$AA?2?$AA?$CF?$AAs?$AA?2?$AA?$CF?$AAs?$AA?2?$AAF?$AAi?$AAl?$AAe?$AAD?$AAe?$AAs?$AAc?$AAr?$AAi?$AAp?$AAt?$AAi?$AAo?$AAn?$AA?$AA@ 100018ec     Pclass.obj
 0001:0000091c       ??_C@_1CG@PJJCHAJ@?$AA?2?$AA?$CF?$AAs?$AA?2?$AA?$CF?$AAs?$AA?2?$AAF?$AAi?$AAl?$AAe?$AAV?$AAe?$AAr?$AAs?$AAi?$AAo?$AAn?$AA?$AA@ 1000191c     Pclass.obj
 0001:00000964       ??_C@_19JHEHLFPM@?$AA?2?$AA?$DP?$AA?$DP?$AA?2?$AA?$AA@ 10001964     Pclass.obj
 0001:00000970       ??_C@_1O@CIJHDDGA@?$AA?$CF?$AAs?$AA?5?$AA?$CF?$AAs?$AA?6?$AA?$AA@ 10001970     Pclass.obj
 0001:00000980       ??_C@_1O@DGEEABED@?$AA?$CF?$AAs?$AA?5?$AA?$CF?$AAd?$AA?6?$AA?$AA@ 10001980     Pclass.obj
 0001:00000990       ??_C@_1M@CBILFCKF@?$AA?5?$AA?$CI?$AA?$CF?$AAs?$AA?$CJ?$AA?$AA@ 10001990     Pclass.obj
 0001:0000099c       ??_C@_17CHCGIDNB@?$AA?$CF?$AAs?$AA?2?$AA?$AA@ 1000199c     Pclass.obj
 0001:000009a4       ??_C@_17GMPJMPF@?$AA?$CF?$AAs?$AA?5?$AA?$AA@ 100019a4     Pclass.obj
 0001:000009ac       ??_C@_1BC@OMEIBLAI@?$AAw?$AAb?$AAe?$AAm?$AAc?$AAo?$AAm?$AAn?$AA?$AA@ 100019ac     Pclass.obj
 0001:000009c0       ??_7PluginEditFieldBinding@@6B@ 100019c0     Pclass.obj
 0001:00000a88       ??_C@_1CM@OLKFIHMK@?$AAN?$AA?0?$AAX?$AA1?$AA5?$AAT?$AA?0?$AAX?$AA1?$AA6?$AAT?$AA?0?$AAX?$AA1?$AA7?$AAT?$AA?0?$AAX?$AA1?$AA8?$AAS?$AA?$AA@ 10001a88     Pclass.obj
 0001:00000ab4       ??_C@_1BG@MNPGDOEP@?$AA1?$AA2?$AA?0?$AA0?$AA?0?$AA0?$AA?0?$AA0?$AA?0?$AA4?$AA?$AA@ 10001ab4     Pclass.obj
 0001:00000acc       ??_C@_1BO@ONCLJEFA@?$AAN?$AA?0?$AAX?$AAI?$AA?0?$AAX?$AAP?$AA?0?$AAX?$AA0?$AAS?$AA?0?$AAX?$AA6?$AA?$AA@ 10001acc     Pclass.obj
 0001:00000aec       ??_C@_1BE@NCGLNDMK@?$AA0?$AA?0?$AA4?$AA?0?$AA2?$AA?0?$AA3?$AA?0?$AA9?$AA?$AA@ 10001aec     Pclass.obj
 0001:00000b00       ??_C@_17KNGPBKAK@?$AAN?$AA?0?$AAN?$AA?$AA@ 10001b00     Pclass.obj
 0001:00000b08       ??_C@_17JPFFEOAH@?$AA0?$AA?0?$AA0?$AA?$AA@ 10001b08     Pclass.obj
 0001:00000b10       ??_C@_1BI@FAMBFJKE@?$AAN?$AA?0?$AAX?$AAI?$AA?0?$AAX?$AAC?$AA?0?$AAD?$AA?0?$AAT?$AA?$AA@ 10001b10     Pclass.obj
 0001:00000b28       ??_C@_1BE@MONBDOED@?$AA0?$AA?0?$AA4?$AA?0?$AA4?$AA?0?$AA0?$AA?0?$AA0?$AA?$AA@ 10001b28     Pclass.obj
 0001:00000b3c       ??_C@_1BG@MICALLFD@?$AAN?$AA?0?$AAX?$AAI?$AA?0?$AAX?$AA4?$AA?0?$AAX?$AA6?$AA?$AA@ 10001b3c     Pclass.obj
 0001:00000b54       ??_C@_1BA@CAEMMMKJ@?$AA0?$AA?0?$AA4?$AA?0?$AA9?$AA?0?$AA9?$AA?$AA@ 10001b54     Pclass.obj
 0001:00000b64       ??_C@_1DI@NKOPFHII@?$AAN?$AA?0?$AAX?$AAI?$AA?0?$AAX?$AA4?$AA?0?$AAX?$AA6?$AA?0?$AAX?$AA1?$AA0?$AA?0?$AAX?$AA1?$AA2?$AA?0?$AAX?$AA0?$AA?0?$AAX?$AA1?$AA?0?$AAX?$AA2?$AA?$AA@ 10001b64     Pclass.obj
 0001:00000b9c       ??_C@_1CG@HGJJIJIH@?$AA1?$AA2?$AA?0?$AA4?$AA?0?$AA0?$AA?0?$AA0?$AA?0?$AA0?$AA?0?$AA0?$AA?0?$AA8?$AA?0?$AA8?$AA?0?$AA8?$AA?$AA@ 10001b9c     Pclass.obj
 0001:00000bc4       ??_C@_19ILLMDDHI@?$AAN?$AA?0?$AAZ?$AAD?$AA?$AA@ 10001bc4     Pclass.obj
 0001:00000bd0       ??_C@_19NMOJBHGD@?$AA1?$AA2?$AA?0?$AA0?$AA?$AA@ 10001bd0     Pclass.obj
 0001:00000be0       ??_C@_1EA@HPDEOPPH@?$AAN?$AA?0?$AAX?$AAP?$AA?0?$AAX?$AA0?$AAS?$AA?0?$AAX?$AA1?$AAS?$AA?0?$AAX?$AA2?$AAS?$AA?0?$AAX?$AA1?$AA1?$AAS?$AA?0?$AAX?$AA1?$AA4?$AAS?$AA?0?$AAX?$AA1?$AA8?$AAS?$AA?$AA@ 10001be0     Pclass.obj
 0001:00000c20       ??_C@_1CA@MGMNHCLL@?$AA0?$AA?0?$AA2?$AA?0?$AA3?$AA?0?$AA2?$AA?0?$AA2?$AA?0?$AA3?$AA?0?$AA4?$AA?0?$AA3?$AA?$AA@ 10001c20     Pclass.obj
 0001:00000c40       ??_C@_1O@JGFFCAGM@?$AAN?$AA?0?$AAX?$AAI?$AA?0?$AAO?$AA?$AA@ 10001c40     Pclass.obj
 0001:00000c50       ??_C@_1O@LAHJLGAL@?$AA0?$AA?0?$AA5?$AA?0?$AA1?$AA5?$AA?$AA@ 10001c50     Pclass.obj
 0001:00000c60       ??_C@_1CC@FANCGEGE@?$AAN?$AA?0?$AAX?$AAI?$AA?0?$AAX?$AAT?$AA?0?$AAX?$AA3?$AA?0?$AAX?$AAG?$AA?0?$AAX?$AAU?$AA?$AA@ 10001c60     Pclass.obj
 0001:00000c84       ??_C@_1BI@DGDJEDOL@?$AA0?$AA?0?$AA4?$AA?0?$AA3?$AA?0?$AA4?$AA?0?$AA4?$AA?0?$AA4?$AA?$AA@ 10001c84     Pclass.obj
 0001:00000c9c       ??_C@_1BG@COBJEPBB@?$AAN?$AA?0?$AAX?$AAI?$AA?0?$AAX?$AAT?$AA?0?$AAX?$AA3?$AA?$AA@ 10001c9c     Pclass.obj
 0001:00000cb4       ??_C@_1BA@EDOGAILM@?$AA0?$AA?0?$AA4?$AA?0?$AA3?$AA?0?$AA4?$AA?$AA@ 10001cb4     Pclass.obj
 0001:00000cc4       ??_C@_15DNHPCDHG@?$AAT?$AAt?$AA?$AA@ 10001cc4     Pclass.obj
 0001:00000ccc       ??_C@_15JOGBDECP@?$AA?0?$AA?5?$AA?$AA@ 10001ccc     Pclass.obj
 0001:00000cd4       ??_C@_1BE@PEGLKBKB@?$AA?6?$AA?$CF?$AAs?$AA?6?$AA?$CF?$AAs?$AA?$CF?$AAs?$AA?6?$AA?$AA@ 10001cd4     Pclass.obj
 0001:00000ce8       ??_C@_1BO@LJMHGFAK@?$AA?$CF?$AA?9?$AA2?$AA2?$AAs?$AA?5?$AA?$CF?$AA0?$AA8?$AAX?$AA?5?$AA?$CF?$AAs?$AA?6?$AA?$AA@ 10001ce8     Pclass.obj
 0001:00000e28       ??_C@_1BE@JKDBKCGH@?$AA?$CF?$AA?9?$AA2?$AA2?$AAs?$AA?5?$AA?$CF?$AAp?$AA?6?$AA?$AA@ 10001e28     Pclass.obj
 0001:00000e3c       ??_C@_1M@NOMFOFMP@?$AAH?$AAW?$AAN?$AAD?$AA?3?$AA?$AA@ 10001e3c     Pclass.obj
 0001:00000e48       ??_C@_1BA@DHHNFIMD@?$AA?6?$AA?$CF?$AAs?$AA?5?$AA?$CF?$AAu?$AA?6?$AA?$AA@ 10001e48     Pclass.obj
 0001:00000e58       ??_C@_1BC@MLKIHIFN@?$AA?6?$AA?$CF?$AAs?$AA?3?$AA?6?$AA?$CF?$AAs?$AA?6?$AA?$AA@ 10001e58     Pclass.obj
 0001:00000e6c       ??_C@_1BG@MDLBKGIE@?$AA?6?$AA?$CF?$AAs?$AA?5?$AA?$CF?$AAs?$AA?5?$AA?$CF?$AAs?$AA?6?$AA?$AA@ 10001e6c     Pclass.obj
 0001:00000e84       ??_C@_1BA@OBCELLNO@?$AA?6?$AA?$CF?$AAs?$AA?5?$AA?$CF?$AAs?$AA?6?$AA?$AA@ 10001e84     Pclass.obj
 0001:00000e94       ??_C@_1O@POMONAHN@?$AA?$CF?$AAs?$AA?5?$AA?$CF?$AAu?$AA?6?$AA?$AA@ 10001e94     Pclass.obj
 0001:00000ea4       ??_C@_1M@LFADDFHG@?$AA?$CF?$AA0?$AA8?$AAX?$AA?6?$AA?$AA@ 10001ea4     Pclass.obj
 0001:00000eb0       ??_C@_17BPBJDALC@?$AA?$CF?$AAu?$AA?6?$AA?$AA@ 10001eb0     Pclass.obj
 0001:00000eb8       ??_C@_1BE@OMBNFFBH@?$AA?$CF?$AAu?$AA?5?$AA?5?$AA?$CI?$AA?$CF?$AAs?$AA?$CJ?$AA?6?$AA?$AA@ 10001eb8     Pclass.obj
 0001:00000ecc       ??_C@_1BC@CLLLJKLA@?$AA?$CF?$AAs?$AA?5?$AA?$CF?$AA0?$AA8?$AAX?$AA?6?$AA?$AA@ 10001ecc     Pclass.obj
 0001:00000ee0       ??_C@_1BC@NEODPHBM@?$AA?$CF?$AAs?$AA?5?$AA?$CF?$AAs?$AA?$CF?$AAs?$AA?6?$AA?$AA@ 10001ee0     Pclass.obj
 0001:00000ef4       ??_C@_1O@CNKEJBH@?$AA?0?$AA?5?$AA?$CF?$AAd?$AA?$CF?$AAs?$AA?$AA@ 10001ef4     Pclass.obj
 0001:00000f1c       ??_C@_19GGNHIDOH@?$AA?4?$AAt?$AAx?$AAt?$AA?$AA@ 10001f1c     Pclass.obj
 0001:00000f28       ??_C@_1BC@OMEIHGFC@?$AAW?$AAS?$AA_?$AAP?$AAO?$AAP?$AAU?$AAP?$AA?$AA@ 10001f28     Pclass.obj
 0001:00000f3c       ??_C@_1BC@ONEEOLLM@?$AAW?$AAS?$AA_?$AAC?$AAH?$AAI?$AAL?$AAD?$AA?$AA@ 10001f3c     Pclass.obj
 0001:00000f50       ??_C@_1BI@GHDIGAD@?$AAW?$AAS?$AA_?$AAM?$AAI?$AAN?$AAI?$AAM?$AAI?$AAZ?$AAE?$AA?$AA@ 10001f50     Pclass.obj
 0001:00000f68       ??_C@_1BG@KLPFHNBP@?$AAW?$AAS?$AA_?$AAV?$AAI?$AAS?$AAI?$AAB?$AAL?$AAE?$AA?$AA@ 10001f68     Pclass.obj
 0001:00000f80       ??_C@_1BI@NKODCGOF@?$AAW?$AAS?$AA_?$AAD?$AAI?$AAS?$AAA?$AAB?$AAL?$AAE?$AAD?$AA?$AA@ 10001f80     Pclass.obj
 0001:00000f98       ??_C@_1CA@PCFJBBHH@?$AAW?$AAS?$AA_?$AAC?$AAL?$AAI?$AAP?$AAS?$AAI?$AAB?$AAL?$AAI?$AAN?$AAG?$AAS?$AA?$AA@ 10001f98     Pclass.obj
 0001:00000fb8       ??_C@_1CA@MPLGGIO@?$AAW?$AAS?$AA_?$AAC?$AAL?$AAI?$AAP?$AAC?$AAH?$AAI?$AAL?$AAD?$AAR?$AAE?$AAN?$AA?$AA@ 10001fb8     Pclass.obj
 0001:00000fd8       ??_C@_1BI@OLBAGOJG@?$AAW?$AAS?$AA_?$AAM?$AAA?$AAX?$AAI?$AAM?$AAI?$AAZ?$AAE?$AA?$AA@ 10001fd8     Pclass.obj
 0001:00000ff0       ??_C@_1BE@DAMMEKNP@?$AAW?$AAS?$AA_?$AAB?$AAO?$AAR?$AAD?$AAE?$AAR?$AA?$AA@ 10001ff0     Pclass.obj
 0001:00001004       ??_C@_1BI@EDHINADK@?$AAW?$AAS?$AA_?$AAD?$AAL?$AAG?$AAF?$AAR?$AAA?$AAM?$AAE?$AA?$AA@ 10002004     Pclass.obj
 0001:0000101c       ??_C@_1BG@CKCLFGFA@?$AAW?$AAS?$AA_?$AAV?$AAS?$AAC?$AAR?$AAO?$AAL?$AAL?$AA?$AA@ 1000201c     Pclass.obj
 0001:00001034       ??_C@_1BG@OMIOJOGF@?$AAW?$AAS?$AA_?$AAH?$AAS?$AAC?$AAR?$AAO?$AAL?$AAL?$AA?$AA@ 10002034     Pclass.obj
 0001:0000104c       ??_C@_1BG@KJOBMDJC@?$AAW?$AAS?$AA_?$AAS?$AAY?$AAS?$AAM?$AAE?$AAN?$AAU?$AA?$AA@ 1000204c     Pclass.obj
 0001:00001064       ??_C@_1BM@GPNNOPCH@?$AAW?$AAS?$AA_?$AAT?$AAH?$AAI?$AAC?$AAK?$AAF?$AAR?$AAA?$AAM?$AAE?$AA?$AA@ 10002064     Pclass.obj
 0001:00001080       ??_C@_1BO@FODKBODI@?$AAW?$AAS?$AA_?$AAM?$AAI?$AAN?$AAI?$AAM?$AAI?$AAZ?$AAE?$AAB?$AAO?$AAX?$AA?$AA@ 10002080     Pclass.obj
 0001:000010a0       ??_C@_1BO@IDJMAOMI@?$AAW?$AAS?$AA_?$AAM?$AAA?$AAX?$AAI?$AAM?$AAI?$AAZ?$AAE?$AAB?$AAO?$AAX?$AA?$AA@ 100020a0     Pclass.obj
 0001:000010c0       ??_C@_1CI@PKBCIOPN@?$AAW?$AAS?$AA_?$AAE?$AAX?$AA_?$AAD?$AAL?$AAG?$AAM?$AAO?$AAD?$AAA?$AAL?$AAF?$AAR?$AAA?$AAM?$AAE?$AA?$AA@ 100020c0     Pclass.obj
 0001:000010e8       ??_C@_1CK@KJECLHMG@?$AAW?$AAS?$AA_?$AAE?$AAX?$AA_?$AAN?$AAO?$AAP?$AAA?$AAR?$AAE?$AAN?$AAT?$AAN?$AAO?$AAT?$AAI?$AAF?$AAY?$AA?$AA@ 100020e8     Pclass.obj
 0001:00001114       ??_C@_1BM@OCBKBALE@?$AAW?$AAS?$AA_?$AAE?$AAX?$AA_?$AAT?$AAO?$AAP?$AAM?$AAO?$AAS?$AAT?$AA?$AA@ 10002114     Pclass.obj
 0001:00001130       ??_C@_1CE@JIDMMICL@?$AAW?$AAS?$AA_?$AAE?$AAX?$AA_?$AAA?$AAC?$AAC?$AAE?$AAP?$AAT?$AAF?$AAI?$AAL?$AAE?$AAS?$AA?$AA@ 10002130     Pclass.obj
 0001:00001154       ??_C@_1CE@PFFPBMCF@?$AAW?$AAS?$AA_?$AAE?$AAX?$AA_?$AAT?$AAR?$AAA?$AAN?$AAS?$AAP?$AAA?$AAR?$AAE?$AAN?$AAT?$AA?$AA@ 10002154     Pclass.obj
 0001:00001178       ??_C@_1BO@MEOEJPLO@?$AAW?$AAS?$AA_?$AAE?$AAX?$AA_?$AAM?$AAD?$AAI?$AAC?$AAH?$AAI?$AAL?$AAD?$AA?$AA@ 10002178     Pclass.obj
 0001:00001198       ??_C@_1CC@IEIGGJGG@?$AAW?$AAS?$AA_?$AAE?$AAX?$AA_?$AAT?$AAO?$AAO?$AAL?$AAW?$AAI?$AAN?$AAD?$AAO?$AAW?$AA?$AA@ 10002198     Pclass.obj
 0001:000011bc       ??_C@_1CC@PLPNIKGL@?$AAW?$AAS?$AA_?$AAE?$AAX?$AA_?$AAW?$AAI?$AAN?$AAD?$AAO?$AAW?$AAE?$AAD?$AAG?$AAE?$AA?$AA@ 100021bc     Pclass.obj
 0001:000011e0       ??_C@_1CC@IAPGCLEG@?$AAW?$AAS?$AA_?$AAE?$AAX?$AA_?$AAC?$AAL?$AAI?$AAE?$AAN?$AAT?$AAE?$AAD?$AAG?$AAE?$AA?$AA@ 100021e0     Pclass.obj
 0001:00001204       ??_C@_1CE@EANKNCIF@?$AAW?$AAS?$AA_?$AAE?$AAX?$AA_?$AAC?$AAO?$AAN?$AAT?$AAE?$AAX?$AAT?$AAH?$AAE?$AAL?$AAP?$AA?$AA@ 10002204     Pclass.obj
 0001:00001228       ??_C@_1BI@GFIADCMK@?$AAW?$AAS?$AA_?$AAE?$AAX?$AA_?$AAR?$AAI?$AAG?$AAH?$AAT?$AA?$AA@ 10002228     Pclass.obj
 0001:00001240       ??_C@_1CC@JOFCJJPB@?$AAW?$AAS?$AA_?$AAE?$AAX?$AA_?$AAR?$AAT?$AAL?$AAR?$AAE?$AAA?$AAD?$AAI?$AAN?$AAG?$AA?$AA@ 10002240     Pclass.obj
 0001:00001264       ??_C@_1CI@EFLDECAB@?$AAW?$AAS?$AA_?$AAE?$AAX?$AA_?$AAL?$AAE?$AAF?$AAT?$AAS?$AAC?$AAR?$AAO?$AAL?$AAL?$AAB?$AAA?$AAR?$AA?$AA@ 10002264     Pclass.obj
 0001:0000128c       ??_C@_1CI@CIFGFFJB@?$AAW?$AAS?$AA_?$AAE?$AAX?$AA_?$AAC?$AAO?$AAN?$AAT?$AAR?$AAO?$AAL?$AAP?$AAA?$AAR?$AAE?$AAN?$AAT?$AA?$AA@ 1000228c     Pclass.obj
 0001:000012b4       ??_C@_1CC@BGEPLDCA@?$AAW?$AAS?$AA_?$AAE?$AAX?$AA_?$AAS?$AAT?$AAA?$AAT?$AAI?$AAC?$AAE?$AAD?$AAG?$AAE?$AA?$AA@ 100022b4     Pclass.obj
 0001:000012d8       ??_C@_1CA@DOAIHHLO@?$AAW?$AAS?$AA_?$AAE?$AAX?$AA_?$AAA?$AAP?$AAP?$AAW?$AAI?$AAN?$AAD?$AAO?$AAW?$AA?$AA@ 100022d8     Pclass.obj
 0001:000012f8       ??_C@_1BM@FAODAMGD@?$AAW?$AAS?$AA_?$AAE?$AAX?$AA_?$AAL?$AAA?$AAY?$AAE?$AAR?$AAE?$AAD?$AA?$AA@ 100022f8     Pclass.obj
 0001:00001314       ??_C@_1CM@DJKNBOGD@?$AAW?$AAS?$AA_?$AAE?$AAX?$AA_?$AAN?$AAO?$AAI?$AAN?$AAH?$AAE?$AAR?$AAI?$AAT?$AAL?$AAA?$AAY?$AAO?$AAU?$AAT?$AA?$AA@ 10002314     Pclass.obj
 0001:00001340       ??_C@_1CA@KMHLBMFI@?$AAW?$AAS?$AA_?$AAE?$AAX?$AA_?$AAL?$AAA?$AAY?$AAO?$AAU?$AAT?$AAR?$AAT?$AAL?$AA?$AA@ 10002340     Pclass.obj
 0001:00001360       ??_C@_1CC@LOFMDOPL@?$AAW?$AAS?$AA_?$AAE?$AAX?$AA_?$AAN?$AAO?$AAA?$AAC?$AAT?$AAI?$AAV?$AAA?$AAT?$AAE?$AA?$AA@ 10002360     Pclass.obj
 0001:00001384       ??_C@_1BC@IALIJCAM@?$AAS?$AAo?$AAr?$AAt?$AAM?$AAo?$AAd?$AAe?$AA?$AA@ 10002384     Pclass.obj
 0001:00001398       ??_C@_1BO@OMKAPLPJ@?$AAS?$AAt?$AAa?$AAr?$AAt?$AAP?$AAa?$AAn?$AAe?$AAl?$AAM?$AAo?$AAd?$AAe?$AA?$AA@ 10002398     Pclass.obj
 0001:000013b8       ??_C@_1M@MOFLFCEC@?$AA?$CF?$AAs?$AA?5?$AA?$CF?$AAs?$AA?$AA@ 100023b8     Pclass.obj
 0001:000013c4       ??_C@_1M@HKFBKEEN@?$AA?$CF?$AA?$CF?$AA?5?$AA?$CF?$AAs?$AA?$AA@ 100023c4     Pclass.obj
 0001:000013e4       ??_C@_15LEKKCGMK@?$AA?2?$AA?2?$AA?$AA@ 100023e4     Pclass.obj
 0001:000013ec       ??_C@_1CK@ECJCGOEK@?$AAP?$AAr?$AAo?$AAc?$AAe?$AAs?$AAs?$AAL?$AAi?$AAs?$AAt?$AA?4?$AAU?$AAs?$AAe?$AAr?$AAn?$AAa?$AAm?$AAe?$AA?$AA@ 100023ec     Pclass.obj
 0001:00001418       ??_C@_1CK@DGKCELDD@?$AAP?$AAr?$AAo?$AAc?$AAe?$AAs?$AAs?$AAL?$AAi?$AAs?$AAt?$AA?4?$AAC?$AAo?$AAm?$AAp?$AAu?$AAt?$AAe?$AAr?$AA?$AA@ 10002418     Pclass.obj
 0001:00001444       ??_C@_1BC@ENICKDH@?$AAC?$AAo?$AAn?$AAt?$AAe?$AAn?$AAt?$AAs?$AA?$AA@ 10002444     Pclass.obj
 0001:00001458       ??_C@_17FJPEEFCB@?$AAp?$AAr?$AAc?$AA?$AA@ 10002458     Pclass.obj
 0001:00001460       ??_C@_15DDHGOCBH@?$AA?4?$AA?4?$AA?$AA@ 10002460     Pclass.obj
 0001:00001468       ??_C@_1DA@BEHINMGJ@?$AAI?$AAO?$AA?5?$AAO?$AAt?$AAh?$AAe?$AAr?$AA?5?$AAO?$AAp?$AAe?$AAr?$AAa?$AAt?$AAi?$AAo?$AAn?$AAs?$AA?1?$AAs?$AAe?$AAc?$AA?$AA@ 10002468     perfthread.obj
 0001:00001498       ??_C@_1DA@HICMAFKK@?$AAI?$AAO?$AA?5?$AAW?$AAr?$AAi?$AAt?$AAe?$AA?5?$AAO?$AAp?$AAe?$AAr?$AAa?$AAt?$AAi?$AAo?$AAn?$AAs?$AA?1?$AAs?$AAe?$AAc?$AA?$AA@ 10002498     perfthread.obj
 0001:000014c8       ??_C@_1CO@LIIKBHDH@?$AAI?$AAO?$AA?5?$AAR?$AAe?$AAa?$AAd?$AA?5?$AAO?$AAp?$AAe?$AAr?$AAa?$AAt?$AAi?$AAo?$AAn?$AAs?$AA?1?$AAs?$AAe?$AAc?$AA?$AA@ 100024c8     perfthread.obj
 0001:000014f8       ??_C@_1CO@LIEOHDCC@?$AAI?$AAO?$AA?5?$AAD?$AAa?$AAt?$AAa?$AA?5?$AAO?$AAp?$AAe?$AAr?$AAa?$AAt?$AAi?$AAo?$AAn?$AAs?$AA?1?$AAs?$AAe?$AAc?$AA?$AA@ 100024f8     perfthread.obj
 0001:00001528       ??_C@_1CG@LBBBPCJA@?$AAI?$AAO?$AA?5?$AAO?$AAt?$AAh?$AAe?$AAr?$AA?5?$AAB?$AAy?$AAt?$AAe?$AAs?$AA?1?$AAs?$AAe?$AAc?$AA?$AA@ 10002528     perfthread.obj
 0001:00001550       ??_C@_1CG@MEJHKKKF@?$AAI?$AAO?$AA?5?$AAW?$AAr?$AAi?$AAt?$AAe?$AA?5?$AAB?$AAy?$AAt?$AAe?$AAs?$AA?1?$AAs?$AAe?$AAc?$AA?$AA@ 10002550     perfthread.obj
 0001:00001578       ??_C@_1CE@EFLEKJAB@?$AAI?$AAO?$AA?5?$AAR?$AAe?$AAa?$AAd?$AA?5?$AAB?$AAy?$AAt?$AAe?$AAs?$AA?1?$AAs?$AAe?$AAc?$AA?$AA@ 10002578     perfthread.obj
 0001:0000159c       ??_C@_1CE@DFDFLLAO@?$AAI?$AAO?$AA?5?$AAD?$AAa?$AAt?$AAa?$AA?5?$AAB?$AAy?$AAt?$AAe?$AAs?$AA?1?$AAs?$AAe?$AAc?$AA?$AA@ 1000259c     perfthread.obj
 0001:000015c0       ??_C@_1CG@KJOKFONA@?$AAV?$AAi?$AAr?$AAt?$AAu?$AAa?$AAl?$AA?5?$AAB?$AAy?$AAt?$AAe?$AAs?$AA?5?$AAP?$AAe?$AAa?$AAk?$AA?$AA@ 100025c0     perfthread.obj
 0001:000015e8       ??_C@_1BM@FMIOMJAE@?$AAV?$AAi?$AAr?$AAt?$AAu?$AAa?$AAl?$AA?5?$AAB?$AAy?$AAt?$AAe?$AAs?$AA?$AA@ 100025e8     perfthread.obj
 0001:00001604       ??_C@_1CA@GADAGCME@?$AAP?$AAa?$AAg?$AAe?$AA?5?$AAF?$AAa?$AAu?$AAl?$AAt?$AAs?$AA?1?$AAs?$AAe?$AAc?$AA?$AA@ 10002604     perfthread.obj
 0001:00001624       ??_C@_1BM@DGDPAMAA@?$AAP?$AAr?$AAi?$AAv?$AAa?$AAt?$AAe?$AA?5?$AAB?$AAy?$AAt?$AAe?$AAs?$AA?$AA@ 10002624     perfthread.obj
 0001:00001640       ??_C@_1CC@IMBAECJF@?$AAP?$AAo?$AAo?$AAl?$AA?5?$AAP?$AAa?$AAg?$AAe?$AAd?$AA?5?$AAB?$AAy?$AAt?$AAe?$AAs?$AA?$AA@ 10002640     perfthread.obj
 0001:00001664       ??_C@_1CI@LLKMGPEG@?$AAP?$AAo?$AAo?$AAl?$AA?5?$AAN?$AAo?$AAn?$AAp?$AAa?$AAg?$AAe?$AAd?$AA?5?$AAB?$AAy?$AAt?$AAe?$AAs?$AA?$AA@ 10002664     perfthread.obj
 0001:0000168c       ??_C@_1CC@OFJLEPCP@?$AAW?$AAo?$AAr?$AAk?$AAi?$AAn?$AAg?$AA?5?$AAS?$AAe?$AAt?$AA?5?$AAP?$AAe?$AAa?$AAk?$AA?$AA@ 1000268c     perfthread.obj
 0001:000016b0       ??_C@_1BI@GCOMDKEO@?$AAW?$AAo?$AAr?$AAk?$AAi?$AAn?$AAg?$AA?5?$AAS?$AAe?$AAt?$AA?$AA@ 100026b0     perfthread.obj
 0001:000016c8       ??_C@_1CK@FGGMBBIH@?$AAP?$AAa?$AAg?$AAe?$AA?5?$AAF?$AAi?$AAl?$AAe?$AA?5?$AAB?$AAy?$AAt?$AAe?$AAs?$AA?5?$AAP?$AAe?$AAa?$AAk?$AA?$AA@ 100026c8     perfthread.obj
 0001:000016f4       ??_C@_1CA@KJMNGIDJ@?$AAP?$AAa?$AAg?$AAe?$AA?5?$AAF?$AAi?$AAl?$AAe?$AA?5?$AAB?$AAy?$AAt?$AAe?$AAs?$AA?$AA@ 100026f4     perfthread.obj
 0001:00001714       ??_C@_1BK@FAAJNJIB@?$AAH?$AAa?$AAn?$AAd?$AAl?$AAe?$AA?5?$AAC?$AAo?$AAu?$AAn?$AAt?$AA?$AA@ 10002714     perfthread.obj
 0001:00001730       ??_C@_1BI@IIOPEKIO@?$AA?$CF?$AA?5?$AAU?$AAs?$AAe?$AAr?$AA?5?$AAT?$AAi?$AAm?$AAe?$AA?$AA@ 10002730     perfthread.obj
 0001:00001748       ??_C@_1CE@FNEMIHOD@?$AA?$CF?$AA?5?$AAP?$AAr?$AAi?$AAv?$AAi?$AAl?$AAe?$AAg?$AAe?$AAd?$AA?5?$AAT?$AAi?$AAm?$AAe?$AA?$AA@ 10002748     perfthread.obj
 0001:0000176c       ??_C@_1CC@DNHMJIKH@?$AA?$CF?$AA?5?$AAP?$AAr?$AAo?$AAc?$AAe?$AAs?$AAs?$AAo?$AAr?$AA?5?$AAT?$AAi?$AAm?$AAe?$AA?$AA@ 1000276c     perfthread.obj
 0001:00001790       ??_C@_19DOGDICKI@?$AA?4?$AAe?$AAx?$AAe?$AA?$AA@ 10002790     perfthread.obj
 0001:0000179c       ??_C@_19DLCFHDFF@?$AAP?$AAE?$AAR?$AAF?$AA?$AA@ 1000279c     perfthread.obj
 0001:000017a8       ??_C@_1BK@IKAFHKBD@?$AAE?$AAl?$AAa?$AAp?$AAs?$AAe?$AAd?$AA?5?$AAT?$AAi?$AAm?$AAe?$AA?$AA@ 100027a8     perfthread.obj
 0001:000017c4       ??_C@_1CI@FNIEMNAI@?$AAC?$AAr?$AAe?$AAa?$AAt?$AAi?$AAn?$AAg?$AA?5?$AAP?$AAr?$AAo?$AAc?$AAe?$AAs?$AAs?$AA?5?$AAI?$AAD?$AA?$AA@ 100027c4     perfthread.obj
 0001:000017ec       ??_C@_1BK@KCHPPKHP@?$AAT?$AAh?$AAr?$AAe?$AAa?$AAd?$AA?5?$AAC?$AAo?$AAu?$AAn?$AAt?$AA?$AA@ 100027ec     perfthread.obj
 0001:00001808       ??_C@_1BM@KCAKLHJN@?$AAP?$AAr?$AAi?$AAo?$AAr?$AAi?$AAt?$AAy?$AA?5?$AAB?$AAa?$AAs?$AAe?$AA?$AA@ 10002808     perfthread.obj
 0001:00001824       ??_C@_1BG@NKNJPBCD@?$AAI?$AAD?$AA?5?$AAP?$AAr?$AAo?$AAc?$AAe?$AAs?$AAs?$AA?$AA@ 10002824     perfthread.obj
 0001:0000183c       ??_C@_1BC@IICCDNLG@?$AAC?$AAo?$AAu?$AAn?$AAt?$AAe?$AAr?$AAs?$AA?$AA@ 1000283c     perfthread.obj
 0001:00001850       ??_C@_1HE@NBDABLAL@?$AAS?$AAo?$AAf?$AAt?$AAw?$AAa?$AAr?$AAe?$AA?2?$AAM?$AAi?$AAc?$AAr?$AAo?$AAs?$AAo?$AAf?$AAt?$AA?2?$AAW?$AAi?$AAn?$AAd?$AAo?$AAw?$AAs?$AA?5?$AAN?$AAT?$AA?2?$AAC?$AAu@ 10002850     perfthread.obj
 0001:000018c4       ??_C@_1CC@DMDJMJLM@?$AAS?$AAe?$AAD?$AAe?$AAb?$AAu?$AAg?$AAP?$AAr?$AAi?$AAv?$AAi?$AAl?$AAe?$AAg?$AAe?$AA?$AA@ 100028c4     Plist.obj
 0001:000018e8       ??_C@_1M@GPDJLPMI@?$AA?4?$AA?$CF?$AA0?$AA3?$AAd?$AA?$AA@ 100028e8     Plist.obj
 0001:000018f4       ??_C@_1CC@EKFMKAAC@?$AA?$CF?$AA1?$AA0?$AA?4?$AA0?$AAf?$AA?5?$AA?5?$AA?$CF?$AA5?$AA?4?$AA0?$AAf?$AA?$CF?$AAs?$AA?6?$AA?$AA@ 100028f4     Plist.obj
 0001:00001918       ??_C@_1BI@HAFBCFCK@?$AA?$CF?$AAs?$AA?5?$AA?$CF?$AA7?$AA?4?$AA0?$AAf?$AA?$CF?$AA?$CF?$AA?6?$AA?$AA@ 10002918     Plist.obj
 0001:00001930       ??_C@_1CG@FOOPEKLK@?$AA?$CF?$AA1?$AA0?$AAI?$AA6?$AA4?$AAu?$AA?5?$AA?5?$AA?$CF?$AA5?$AAI?$AA6?$AA4?$AAu?$AA?$CF?$AAs?$AA?6?$AA?$AA@ 10002930     Plist.obj
 0001:00001958       ??_C@_1BC@CIAMCHCM@?$AA?$CF?$AA1?$AA0?$AAI?$AA6?$AA4?$AAu?$AA?6?$AA?$AA@ 10002958     Plist.obj
 0001:0000196c       ??_C@_1BA@DJJLONDK@?$AA?$CF?$AA1?$AA0?$AA?4?$AA0?$AAf?$AA?6?$AA?$AA@ 1000296c     Plist.obj
 0001:0000197c       ??_C@_1O@KBBIJFEI@?$AA?$CF?$AA?9?$AA2?$AA4?$AAs?$AA?5?$AA?$AA@ 1000297c     Plist.obj
 0001:0000198c       ??_C@_13EBCNDICG@?$AA?3?$AA?$AA@ 1000298c     Plist.obj
 0001:00001990       ??_C@_17MJEANDKP@?$AA?$CF?$AAs?$AA?6?$AA?$AA@ 10002990     Plist.obj
 0001:00001998       ??_C@_19FJPIAKGM@?$AA?$CF?$AAs?$AA?6?$AA?6?$AA?$AA@ 10002998     Plist.obj
 0001:000019a4       ??_C@_1BA@LFJAMCEC@?$AA?$CF?$AAs?$AA?5?$AA?$CF?$AAs?$AA?6?$AA?6?$AA?$AA@ 100029a4     Plist.obj
 0001:000019b4       ??_C@_17ENEANJDH@?$AA?5?$AA?$CF?$AAs?$AA?$AA@ 100029b4     Plist.obj
 0001:000019bc       ??_C@_1BE@KPJOOIA@?$AA?5?$AA?5?$AA?$CF?$AAp?$AA?5?$AA?5?$AA?$CF?$AA6?$AAX?$AA?$AA@ 100029bc     Plist.obj
 0001:000019d0       ??_C@_15JNBOKNOG@?$AA?$AN?$AA?6?$AA?$AA@ 100029d0     Pmix.obj
 0001:000019d8       ??_C@_1BG@FFJGBKCB@?$AAE?$AAr?$AAr?$AAo?$AAr?$AA?5?$AA0?$AAx?$AA?$CF?$AAx?$AA?$AA@ 100029d8     Pmix.obj
 0001:000019f0       _IID_IWbemLocator          100029f0     WMI.obj
 0001:00001a00       _CLSID_WbemLocator         10002a00     WMI.obj
 0001:00001a10       ??_C@_1DA@BIBEJFMF@?$AAW?$AAi?$AAn?$AA3?$AA2?$AA_?$AAP?$AAr?$AAo?$AAc?$AAe?$AAs?$AAs?$AA?4?$AAH?$AAa?$AAn?$AAd?$AAl?$AAe?$AA?$DN?$AA?$CF?$AAu?$AA?$AA@ 10002a10     WMI.obj
 0001:00001a40       ??_C@_1BO@CLCOBGDE@?$AAE?$AAx?$AAe?$AAc?$AAu?$AAt?$AAa?$AAb?$AAl?$AAe?$AAP?$AAa?$AAt?$AAh?$AA?$AA@ 10002a40     WMI.obj
 0001:00001a60       ??_C@_1BC@JHNNEHFE@?$AAP?$AAr?$AAi?$AAo?$AAr?$AAi?$AAt?$AAy?$AA?$AA@ 10002a60     WMI.obj
 0001:00001a74       ??_C@_1O@OAMNPMOM@?$AAD?$AAo?$AAm?$AAa?$AAi?$AAn?$AA?$AA@ 10002a74     WMI.obj
 0001:00001a84       ??_C@_19PIJILKAI@?$AAU?$AAs?$AAe?$AAr?$AA?$AA@ 10002a84     WMI.obj
 0001:00001a90       ??_C@_1BC@HJJANEGO@?$AAG?$AAe?$AAt?$AAO?$AAw?$AAn?$AAe?$AAr?$AA?$AA@ 10002a90     WMI.obj
 0001:00001aa4       ??_C@_17NKMLOKHF@?$AAS?$AAi?$AAd?$AA?$AA@ 10002aa4     WMI.obj
 0001:00001aac       ??_C@_1BI@OIPNMPCL@?$AAG?$AAe?$AAt?$AAO?$AAw?$AAn?$AAe?$AAr?$AAS?$AAi?$AAd?$AA?$AA@ 10002aac     WMI.obj
 0001:00001ac4       ??_C@_1BE@CFEJJKFE@?$AAS?$AAe?$AAs?$AAs?$AAi?$AAo?$AAn?$AAI?$AAd?$AA?$AA@ 10002ac4     WMI.obj
 0001:00001ad8       ??_C@_1BI@FLOHINJE@?$AAR?$AAe?$AAt?$AAu?$AAr?$AAn?$AAV?$AAa?$AAl?$AAu?$AAe?$AA?$AA@ 10002ad8     WMI.obj
 0001:00001af0       ??_C@_1BM@MLGLIGHJ@?$AAW?$AAi?$AAn?$AA3?$AA2?$AA_?$AAP?$AAr?$AAo?$AAc?$AAe?$AAs?$AAs?$AA?$AA@ 10002af0     WMI.obj
 0001:00001b0c       ??_C@_1BI@NKNJJIDM@?$AAS?$AAe?$AAt?$AAP?$AAr?$AAi?$AAo?$AAr?$AAi?$AAt?$AAy?$AA?$AA@ 10002b0c     WMI.obj
 0001:00001b24       ??_C@_1BE@PBPGMODO@?$AAT?$AAe?$AAr?$AAm?$AAi?$AAn?$AAa?$AAt?$AAe?$AA?$AA@ 10002b24     WMI.obj
 0001:00001b38       ??_C@_1O@GGHBFGJC@?$AAR?$AAe?$AAa?$AAs?$AAo?$AAn?$AA?$AA@ 10002b38     WMI.obj
 0001:00001b48       ??_C@_1CA@ECJNGEII@?$AA?2?$AA?2?$AA?$CF?$AAs?$AA?2?$AAr?$AAo?$AAo?$AAt?$AA?2?$AAc?$AAi?$AAm?$AAv?$AA2?$AA?$AA@ 10002b48     WMI.obj
 0001:00001b68       ??_C@_13JOFGPIOO@?$AA?4?$AA?$AA@ 10002b68     WMI.obj
 0001:00001b6c       _MainGuid                  10002b6c     Proclist.obj
 0001:00001b7c       _MenuGuid                  10002b7c     Proclist.obj
 0001:00001b8c       _ConfigDialogGuid          10002b8c     Proclist.obj
 0001:00001b9c       ??_C@_0BC@IOEGILCE@CoSetProxyBlanket?$AA@ 10002b9c     Proclist.obj
 0001:00001bb0       ??_C@_1M@FFPAMFOB@?$AAo?$AAl?$AAe?$AA3?$AA2?$AA?$AA@ 10002bb0     Proclist.obj
 0001:00001bbc       ??_C@_0BA@FKGDNIJG@GetGuiResources?$AA@ 10002bbc     Proclist.obj
 0001:00001bcc       ??_C@_1O@BCCLBEOE@?$AAu?$AAs?$AAe?$AAr?$AA3?$AA2?$AA?$AA@ 10002bcc     Proclist.obj
 0001:00001bdc       ??_C@_0BD@MCBOPCDK@LookupAccountNameW?$AA@ 10002bdc     Proclist.obj
 0001:00001bf0       ??_C@_0BD@LMGFHOAE@GetSidSubAuthority?$AA@ 10002bf0     Proclist.obj
 0001:00001c04       ??_C@_0BI@LPFJALDI@GetSidSubAuthorityCount?$AA@ 10002c04     Proclist.obj
 0001:00001c1c       ??_C@_0BK@FIHGNING@GetSidIdentifierAuthority?$AA@ 10002c1c     Proclist.obj
 0001:00001c38       ??_C@_0L@KJHKJIPF@IsValidSid?$AA@ 10002c38     Proclist.obj
 0001:00001c44       ??_C@_1BC@DNHGCMLG@?$AAa?$AAd?$AAv?$AAa?$AAp?$AAi?$AA3?$AA2?$AA?$AA@ 10002c44     Proclist.obj
 0001:00001c58       ??_C@_0P@LKABJJMO@IsWow64Process?$AA@ 10002c58     Proclist.obj
 0001:00001c68       ??_C@_1BC@GDMECMAK@?$AAk?$AAe?$AAr?$AAn?$AAe?$AAl?$AA3?$AA2?$AA?$AA@ 10002c68     Proclist.obj
 0001:00001c7c       ??_C@_0BH@DLPGICA@NtQueryInformationFile?$AA@ 10002c7c     Proclist.obj
 0001:00001c94       ??_C@_0BJ@NDLOPGCH@NtQuerySystemInformation?$AA@ 10002c94     Proclist.obj
 0001:00001cb0       ??_C@_0O@IFMDHOMC@NtQueryObject?$AA@ 10002cb0     Proclist.obj
 0001:00001cc0       ??_C@_0BJ@HKKELGGC@NtQueryInformationThread?$AA@ 10002cc0     Proclist.obj
 0001:00001cdc       ??_C@_0BK@EGDDIFMK@NtQueryInformationProcess?$AA@ 10002cdc     Proclist.obj
 0001:00001cf8       ??_C@_1M@OAIMIKLP@?$AAn?$AAt?$AAd?$AAl?$AAl?$AA?$AA@ 10002cf8     Proclist.obj
 0001:00001d04       ??_C@_1DE@BGKMIKPD@?$AAE?$AAu?$AAg?$AAe?$AAn?$AAe?$AA?5?$AAR?$AAo?$AAs?$AAh?$AAa?$AAl?$AA?5?$AA?$CG?$AA?5?$AAF?$AAa?$AAr?$AA?5?$AAG?$AAr?$AAo?$AAu?$AAp?$AA?$AA@ 10002d04     Proclist.obj
 0001:00001d38       ??_C@_1DK@DCAMPEPJ@?$AAP?$AAr?$AAo?$AAc?$AAe?$AAs?$AAs?$AA?5?$AAL?$AAi?$AAs?$AAt?$AA?5?$AAf?$AAo?$AAr?$AA?5?$AAF?$AAA?$AAR?$AA?5?$AAM?$AAa?$AAn?$AAa?$AAg?$AAe?$AAr?$AA?$AA@ 10002d38     Proclist.obj
 0001:00001d74       ??_C@_1BC@PDEABLIN@?$AAP?$AAr?$AAo?$AAc?$AAL?$AAi?$AAs?$AAt?$AA?$AA@ 10002d74     Proclist.obj
 0001:00001d88       ??_C@_1M@MNPEKPKO@?$AAp?$AAl?$AAi?$AAs?$AAt?$AA?$AA@ 10002d88     Proclist.obj
 0001:00001da0       __imp__EncodePointer@4     10002da0     vc_crt_fix.obj
 0001:00001da4       __imp__DecodePointer@4     10002da4     vc_crt_fix.obj
 0001:00001da8       __imp__GetModuleHandleExW@12 10002da8     vc_crt_fix.obj
 0001:00001dc0       ??_C@_0O@NLDKAIKN@EncodePointer?$AA@ 10002dc0     vc_crt_fix_impl.obj
 0001:00001dd0       ??_C@_0O@KBPMFGHI@DecodePointer?$AA@ 10002dd0     vc_crt_fix_impl.obj
 0001:00001de0       ??_C@_0BD@GIGEJCNH@GetModuleHandleExW?$AA@ 10002de0     vc_crt_fix_impl.obj
 0001:00001df8       ??_7bad_alloc@std@@6B@     10002df8     LIBCMT:new.obj
 0001:00001e00       ??_C@_0P@GHFPNOJB@bad?5allocation?$AA@ 10002e00     LIBCMT:new.obj
 0001:00001e10       __FPinit                   10002e10     LIBCMT:_fpinit_.obj
 0001:00001e14       __pRawDllMain              10002e14     LIBCMT:dllcrt0.obj
 0001:00001e14       __pDefaultRawDllMain       10002e14     LIBCMT:dllcrt0.obj
 0001:00001e18       ??_C@_1BC@GDGBMEMK@?$AAH?$AAH?$AA?3?$AAm?$AAm?$AA?3?$AAs?$AAs?$AA?$AA@ 10002e18     LIBCMT:nlsdata2.obj
 0001:00001e2c       ??_C@_1CI@KNAKOEBC@?$AAd?$AAd?$AAd?$AAd?$AA?0?$AA?5?$AAM?$AAM?$AAM?$AAM?$AA?5?$AAd?$AAd?$AA?0?$AA?5?$AAy?$AAy?$AAy?$AAy?$AA?$AA@ 10002e2c     LIBCMT:nlsdata2.obj
 0001:00001e54       ??_C@_1BC@IEBCMHCM@?$AAM?$AAM?$AA?1?$AAd?$AAd?$AA?1?$AAy?$AAy?$AA?$AA@ 10002e54     LIBCMT:nlsdata2.obj
 0001:00001e68       ??_C@_15CLMNNGEL@?$AAP?$AAM?$AA?$AA@ 10002e68     LIBCMT:nlsdata2.obj
 0001:00001e70       ??_C@_15ODEHAHHF@?$AAA?$AAM?$AA?$AA@ 10002e70     LIBCMT:nlsdata2.obj
 0001:00001e78       ??_C@_1BC@FEMKIFH@?$AAD?$AAe?$AAc?$AAe?$AAm?$AAb?$AAe?$AAr?$AA?$AA@ 10002e78     LIBCMT:nlsdata2.obj
 0001:00001e8c       ??_C@_1BC@BGLIFPF@?$AAN?$AAo?$AAv?$AAe?$AAm?$AAb?$AAe?$AAr?$AA?$AA@ 10002e8c     LIBCMT:nlsdata2.obj
 0001:00001ea0       ??_C@_1BA@EPANDLNG@?$AAO?$AAc?$AAt?$AAo?$AAb?$AAe?$AAr?$AA?$AA@ 10002ea0     LIBCMT:nlsdata2.obj
 0001:00001eb0       ??_C@_1BE@DKAAMBJL@?$AAS?$AAe?$AAp?$AAt?$AAe?$AAm?$AAb?$AAe?$AAr?$AA?$AA@ 10002eb0     LIBCMT:nlsdata2.obj
 0001:00001ec4       ??_C@_1O@PAHLKOAC@?$AAA?$AAu?$AAg?$AAu?$AAs?$AAt?$AA?$AA@ 10002ec4     LIBCMT:nlsdata2.obj
 0001:00001ed4       ??_C@_19BIFMLPCD@?$AAJ?$AAu?$AAl?$AAy?$AA?$AA@ 10002ed4     LIBCMT:nlsdata2.obj
 0001:00001ee0       ??_C@_19EPFLPGAP@?$AAJ?$AAu?$AAn?$AAe?$AA?$AA@ 10002ee0     LIBCMT:nlsdata2.obj
 0001:00001eec       ??_C@_1M@GJNLMHFD@?$AAA?$AAp?$AAr?$AAi?$AAl?$AA?$AA@ 10002eec     LIBCMT:nlsdata2.obj
 0001:00001ef8       ??_C@_1M@IKEENEDF@?$AAM?$AAa?$AAr?$AAc?$AAh?$AA?$AA@ 10002ef8     LIBCMT:nlsdata2.obj
 0001:00001f04       ??_C@_1BC@JGDDFFAM@?$AAF?$AAe?$AAb?$AAr?$AAu?$AAa?$AAr?$AAy?$AA?$AA@ 10002f04     LIBCMT:nlsdata2.obj
 0001:00001f18       ??_C@_1BA@EFMEIEBA@?$AAJ?$AAa?$AAn?$AAu?$AAa?$AAr?$AAy?$AA?$AA@ 10002f18     LIBCMT:nlsdata2.obj
 0001:00001f28       ??_C@_17EGKACKIF@?$AAD?$AAe?$AAc?$AA?$AA@ 10002f28     LIBCMT:nlsdata2.obj
 0001:00001f30       ??_C@_17BBDMLCIG@?$AAN?$AAo?$AAv?$AA?$AA@ 10002f30     LIBCMT:nlsdata2.obj
 0001:00001f38       ??_C@_17FNLKOI@?$AAO?$AAc?$AAt?$AA?$AA@ 10002f38     LIBCMT:nlsdata2.obj
 0001:00001f40       ??_C@_17HCHCOKMG@?$AAS?$AAe?$AAp?$AA?$AA@ 10002f40     LIBCMT:nlsdata2.obj
 0001:00001f48       ??_C@_17ICPELBCN@?$AAA?$AAu?$AAg?$AA?$AA@ 10002f48     LIBCMT:nlsdata2.obj
 0001:00001f50       ??_C@_17IJPCKHK@?$AAJ?$AAu?$AAl?$AA?$AA@ 10002f50     LIBCMT:nlsdata2.obj
 0001:00001f58       ??_C@_17KCJGOCPB@?$AAJ?$AAu?$AAn?$AA?$AA@ 10002f58     LIBCMT:nlsdata2.obj
 0001:00001f60       ??_C@_17PNNKMEED@?$AAM?$AAa?$AAy?$AA?$AA@ 10002f60     LIBCMT:nlsdata2.obj
 0001:00001f68       ??_C@_17LFPOIHDD@?$AAA?$AAp?$AAr?$AA?$AA@ 10002f68     LIBCMT:nlsdata2.obj
 0001:00001f70       ??_C@_17CKNLEDEC@?$AAM?$AAa?$AAr?$AA?$AA@ 10002f70     LIBCMT:nlsdata2.obj
 0001:00001f78       ??_C@_17LMDJEKJN@?$AAF?$AAe?$AAb?$AA?$AA@ 10002f78     LIBCMT:nlsdata2.obj
 0001:00001f80       ??_C@_17DKNBKCHM@?$AAJ?$AAa?$AAn?$AA?$AA@ 10002f80     LIBCMT:nlsdata2.obj
 0001:00001f88       ??_C@_1BC@ENMNNPAJ@?$AAS?$AAa?$AAt?$AAu?$AAr?$AAd?$AAa?$AAy?$AA?$AA@ 10002f88     LIBCMT:nlsdata2.obj
 0001:00001f9c       ??_C@_1O@PDICJHAG@?$AAF?$AAr?$AAi?$AAd?$AAa?$AAy?$AA?$AA@ 10002f9c     LIBCMT:nlsdata2.obj
 0001:00001fac       ??_C@_1BC@HHMNLIHE@?$AAT?$AAh?$AAu?$AAr?$AAs?$AAd?$AAa?$AAy?$AA?$AA@ 10002fac     LIBCMT:nlsdata2.obj
 0001:00001fc0       ??_C@_1BE@EBOGMDOH@?$AAW?$AAe?$AAd?$AAn?$AAe?$AAs?$AAd?$AAa?$AAy?$AA?$AA@ 10002fc0     LIBCMT:nlsdata2.obj
 0001:00001fd4       ??_C@_1BA@ENFBFFEK@?$AAT?$AAu?$AAe?$AAs?$AAd?$AAa?$AAy?$AA?$AA@ 10002fd4     LIBCMT:nlsdata2.obj
 0001:00001fe4       ??_C@_1O@MMNBFLIA@?$AAM?$AAo?$AAn?$AAd?$AAa?$AAy?$AA?$AA@ 10002fe4     LIBCMT:nlsdata2.obj
 0001:00001ff4       ??_C@_1O@IHNHDHPB@?$AAS?$AAu?$AAn?$AAd?$AAa?$AAy?$AA?$AA@ 10002ff4     LIBCMT:nlsdata2.obj
 0001:00002004       ??_C@_17GGIBDPIH@?$AAS?$AAa?$AAt?$AA?$AA@ 10003004     LIBCMT:nlsdata2.obj
 0001:0000200c       ??_C@_17HFOLPPLP@?$AAF?$AAr?$AAi?$AA?$AA@ 1000300c     LIBCMT:nlsdata2.obj
 0001:00002014       ??_C@_17PDPHAADD@?$AAT?$AAh?$AAu?$AA?$AA@ 10003014     LIBCMT:nlsdata2.obj
 0001:0000201c       ??_C@_17CJEDCEPE@?$AAW?$AAe?$AAd?$AA?$AA@ 1000301c     LIBCMT:nlsdata2.obj
 0001:00002024       ??_C@_17BMKGEGOJ@?$AAT?$AAu?$AAe?$AA?$AA@ 10003024     LIBCMT:nlsdata2.obj
 0001:0000202c       ??_C@_17KBOMKBF@?$AAM?$AAo?$AAn?$AA?$AA@ 1000302c     LIBCMT:nlsdata2.obj
 0001:00002034       ??_C@_17MBGCMIPB@?$AAS?$AAu?$AAn?$AA?$AA@ 10003034     LIBCMT:nlsdata2.obj
 0001:0000203c       ??_C@_08JCCMCCIL@HH?3mm?3ss?$AA@ 1000303c     LIBCMT:nlsdata2.obj
 0001:00002048       ??_C@_0BE@CKGJFCPC@dddd?0?5MMMM?5dd?0?5yyyy?$AA@ 10003048     LIBCMT:nlsdata2.obj
 0001:0000205c       ??_C@_08BPBNCDIB@MM?1dd?1yy?$AA@ 1000305c     LIBCMT:nlsdata2.obj
 0001:00002068       ??_C@_02CJNFDJBF@PM?$AA@   10003068     LIBCMT:nlsdata2.obj
 0001:0000206c       ??_C@_02DEDBPAFC@AM?$AA@   1000306c     LIBCMT:nlsdata2.obj
 0001:00002070       ??_C@_08EDHMEBNP@December?$AA@ 10003070     LIBCMT:nlsdata2.obj
 0001:0000207c       ??_C@_08HCHEGEOA@November?$AA@ 1000307c     LIBCMT:nlsdata2.obj
 0001:00002088       ??_C@_07JJNFCEND@October?$AA@ 10003088     LIBCMT:nlsdata2.obj
 0001:00002090       ??_C@_09BHHEALKD@September?$AA@ 10003090     LIBCMT:nlsdata2.obj
 0001:0000209c       ??_C@_06LBBHFDDG@August?$AA@ 1000309c     LIBCMT:nlsdata2.obj
 0001:000020a4       ??_C@_04MIEPOIFP@July?$AA@ 100030a4     LIBCMT:nlsdata2.obj
 0001:000020ac       ??_C@_04CNLMGBGM@June?$AA@ 100030ac     LIBCMT:nlsdata2.obj
 0001:000020b4       ??_C@_05DMJDNLEJ@April?$AA@ 100030b4     LIBCMT:nlsdata2.obj
 0001:000020bc       ??_C@_05HPCKOFNC@March?$AA@ 100030bc     LIBCMT:nlsdata2.obj
 0001:000020c4       ??_C@_08GNJGEPFN@February?$AA@ 100030c4     LIBCMT:nlsdata2.obj
 0001:000020d0       ??_C@_07CGJPFGJA@January?$AA@ 100030d0     LIBCMT:nlsdata2.obj
 0001:000020d8       ??_C@_03MKABNOCG@Dec?$AA@  100030d8     LIBCMT:nlsdata2.obj
 0001:000020dc       ??_C@_03JPJOFNIA@Nov?$AA@  100030dc     LIBCMT:nlsdata2.obj
 0001:000020e0       ??_C@_03BMAOKBAD@Oct?$AA@  100030e0     LIBCMT:nlsdata2.obj
 0001:000020e4       ??_C@_03GGCAPAJC@Sep?$AA@  100030e4     LIBCMT:nlsdata2.obj
 0001:000020e8       ??_C@_03IFJFEIGA@Aug?$AA@  100030e8     LIBCMT:nlsdata2.obj
 0001:000020ec       ??_C@_03LBGABGKK@Jul?$AA@  100030ec     LIBCMT:nlsdata2.obj
 0001:000020f0       ??_C@_03IDFGHECI@Jun?$AA@  100030f0     LIBCMT:nlsdata2.obj
 0001:000020f4       ??_C@_03CNMDKL@May?$AA@    100030f4     LIBCMT:nlsdata2.obj
 0001:000020f8       ??_C@_03LEOLGMJP@Apr?$AA@  100030f8     LIBCMT:nlsdata2.obj
 0001:000020fc       ??_C@_03ODNJBKGA@Mar?$AA@  100030fc     LIBCMT:nlsdata2.obj
 0001:00002100       ??_C@_03HJBDCHOM@Feb?$AA@  10003100     LIBCMT:nlsdata2.obj
 0001:00002104       ??_C@_03JIHJHPIE@Jan?$AA@  10003104     LIBCMT:nlsdata2.obj
 0001:00002108       ??_C@_08INBOOONO@Saturday?$AA@ 10003108     LIBCMT:nlsdata2.obj
 0001:00002114       ??_C@_06JECMNKMI@Friday?$AA@ 10003114     LIBCMT:nlsdata2.obj
 0001:0000211c       ??_C@_08HACCIKIA@Thursday?$AA@ 1000311c     LIBCMT:nlsdata2.obj
 0001:00002128       ??_C@_09DLIGFAKA@Wednesday?$AA@ 10003128     LIBCMT:nlsdata2.obj
 0001:00002134       ??_C@_07BAAGCFCM@Tuesday?$AA@ 10003134     LIBCMT:nlsdata2.obj
 0001:0000213c       ??_C@_06JLEDEDGH@Monday?$AA@ 1000313c     LIBCMT:nlsdata2.obj
 0001:00002144       ??_C@_06OOPIFAJ@Sunday?$AA@ 10003144     LIBCMT:nlsdata2.obj
 0001:0000214c       ??_C@_03FEFJNEK@Sat?$AA@   1000314c     LIBCMT:nlsdata2.obj
 0001:00002150       ??_C@_03IDIOELNC@Fri?$AA@  10003150     LIBCMT:nlsdata2.obj
 0001:00002154       ??_C@_03IOFIKPDN@Thu?$AA@  10003154     LIBCMT:nlsdata2.obj
 0001:00002158       ??_C@_03MHOMLAJA@Wed?$AA@  10003158     LIBCMT:nlsdata2.obj
 0001:0000215c       ??_C@_03NAGEINEP@Tue?$AA@  1000315c     LIBCMT:nlsdata2.obj
 0001:00002160       ??_C@_03PDAGKDH@Mon?$AA@   10003160     LIBCMT:nlsdata2.obj
 0001:00002164       ??_C@_03KOEHGMDN@Sun?$AA@  10003164     LIBCMT:nlsdata2.obj
 0001:00002168       ??_C@_1BK@DBDEIDLH@?$AAK?$AAE?$AAR?$AAN?$AAE?$AAL?$AA3?$AA2?$AA?4?$AAD?$AAL?$AAL?$AA?$AA@ 10003168     LIBCMT:tidtable.obj
 0001:00002184       ??_C@_07PEJMOBNF@FlsFree?$AA@ 10003184     LIBCMT:tidtable.obj
 0001:0000218c       ??_C@_0M@JCPCPOEF@FlsSetValue?$AA@ 1000318c     LIBCMT:tidtable.obj
 0001:00002198       ??_C@_0M@GDNOONDI@FlsGetValue?$AA@ 10003198     LIBCMT:tidtable.obj
 0001:000021a4       ??_C@_08KNHFBNJ@FlsAlloc?$AA@ 100031a4     LIBCMT:tidtable.obj
 0001:00002230       ??_C@_01NEMOKFLO@?$DN?$AA@ 10003230     LIBCMT:setlocal.obj
 0001:00002232       ??_C@_00CNPNBAHC@?$AA@     10003232     LIBCMT:setlocal.obj
 0001:00002234       ??_C@_0P@MIGLKIOC@CorExitProcess?$AA@ 10003234     LIBCMT:crt0dat.obj
 0001:00002244       ??_C@_1BI@BGOHAHKC@?$AAm?$AAs?$AAc?$AAo?$AAr?$AAe?$AAe?$AA?4?$AAd?$AAl?$AAl?$AA?$AA@ 10003244     LIBCMT:crt0dat.obj
 0001:0000225c       ??_C@_1BO@BKOMIGKJ@?$AAr?$AAu?$AAn?$AAt?$AAi?$AAm?$AAe?$AA?5?$AAe?$AAr?$AAr?$AAo?$AAr?$AA?5?$AA?$AA@ 1000325c     LIBCMT:crt0msg.obj
 0001:0000227c       ??_C@_1BM@JBBEPPHI@?$AAT?$AAL?$AAO?$AAS?$AAS?$AA?5?$AAe?$AAr?$AAr?$AAo?$AAr?$AA?$AN?$AA?6?$AA?$AA@ 1000327c     LIBCMT:crt0msg.obj
 0001:00002298       ??_C@_1BK@KMOMNAAI@?$AAS?$AAI?$AAN?$AAG?$AA?5?$AAe?$AAr?$AAr?$AAo?$AAr?$AA?$AN?$AA?6?$AA?$AA@ 10003298     LIBCMT:crt0msg.obj
 0001:000022b4       ??_C@_1BO@BFCDCGC@?$AAD?$AAO?$AAM?$AAA?$AAI?$AAN?$AA?5?$AAe?$AAr?$AAr?$AAo?$AAr?$AA?$AN?$AA?6?$AA?$AA@ 100032b4     LIBCMT:crt0msg.obj
 0001:000022d8       ??_C@_1BOO@KGEDBGAJ@?$AAR?$AA6?$AA0?$AA3?$AA3?$AA?$AN?$AA?6?$AA?9?$AA?5?$AAA?$AAt?$AAt?$AAe?$AAm?$AAp?$AAt?$AA?5?$AAt?$AAo?$AA?5?$AAu?$AAs?$AAe?$AA?5?$AAM?$AAS?$AAI?$AAL?$AA?5?$AAc?$AAo?$AAd@ 100032d8     LIBCMT:crt0msg.obj
 0001:000024c8       ??_C@_1GG@GOPILAJP@?$AAR?$AA6?$AA0?$AA3?$AA2?$AA?$AN?$AA?6?$AA?9?$AA?5?$AAn?$AAo?$AAt?$AA?5?$AAe?$AAn?$AAo?$AAu?$AAg?$AAh?$AA?5?$AAs?$AAp?$AAa?$AAc?$AAe?$AA?5?$AAf?$AAo?$AAr?$AA?5?$AAl?$AAo@ 100034c8     LIBCMT:crt0msg.obj
 0001:00002530       ??_C@_1MG@ENCOOIDF@?$AAR?$AA6?$AA0?$AA3?$AA1?$AA?$AN?$AA?6?$AA?9?$AA?5?$AAA?$AAt?$AAt?$AAe?$AAm?$AAp?$AAt?$AA?5?$AAt?$AAo?$AA?5?$AAi?$AAn?$AAi?$AAt?$AAi?$AAa?$AAl?$AAi?$AAz?$AAe?$AA?5?$AAt@ 10003530     LIBCMT:crt0msg.obj
 0001:000025f8       ??_C@_1DO@BMFCDCD@?$AAR?$AA6?$AA0?$AA3?$AA0?$AA?$AN?$AA?6?$AA?9?$AA?5?$AAC?$AAR?$AAT?$AA?5?$AAn?$AAo?$AAt?$AA?5?$AAi?$AAn?$AAi?$AAt?$AAi?$AAa?$AAl?$AAi?$AAz?$AAe?$AAd?$AA?$AN?$AA?6?$AA?$AA@ 100035f8     LIBCMT:crt0msg.obj
 0001:00002638       ??_C@_1EK@HHFLMAOL@?$AAR?$AA6?$AA0?$AA2?$AA8?$AA?$AN?$AA?6?$AA?9?$AA?5?$AAu?$AAn?$AAa?$AAb?$AAl?$AAe?$AA?5?$AAt?$AAo?$AA?5?$AAi?$AAn?$AAi?$AAt?$AAi?$AAa?$AAl?$AAi?$AAz?$AAe?$AA?5?$AAh?$AAe@ 10003638     LIBCMT:crt0msg.obj
 0001:00002688       ??_C@_1GK@MFGOKLAG@?$AAR?$AA6?$AA0?$AA2?$AA7?$AA?$AN?$AA?6?$AA?9?$AA?5?$AAn?$AAo?$AAt?$AA?5?$AAe?$AAn?$AAo?$AAu?$AAg?$AAh?$AA?5?$AAs?$AAp?$AAa?$AAc?$AAe?$AA?5?$AAf?$AAo?$AAr?$AA?5?$AAl?$AAo@ 10003688     LIBCMT:crt0msg.obj
 0001:000026f8       ??_C@_1GK@MCAAGJMO@?$AAR?$AA6?$AA0?$AA2?$AA6?$AA?$AN?$AA?6?$AA?9?$AA?5?$AAn?$AAo?$AAt?$AA?5?$AAe?$AAn?$AAo?$AAu?$AAg?$AAh?$AA?5?$AAs?$AAp?$AAa?$AAc?$AAe?$AA?5?$AAf?$AAo?$AAr?$AA?5?$AAs?$AAt@ 100036f8     LIBCMT:crt0msg.obj
 0001:00002768       ??_C@_1EM@MAADIHMB@?$AAR?$AA6?$AA0?$AA2?$AA5?$AA?$AN?$AA?6?$AA?9?$AA?5?$AAp?$AAu?$AAr?$AAe?$AA?5?$AAv?$AAi?$AAr?$AAt?$AAu?$AAa?$AAl?$AA?5?$AAf?$AAu?$AAn?$AAc?$AAt?$AAi?$AAo?$AAn?$AA?5?$AAc@ 10003768     LIBCMT:crt0msg.obj
 0001:000027b8       ??_C@_1GK@FHCKBEFA@?$AAR?$AA6?$AA0?$AA2?$AA4?$AA?$AN?$AA?6?$AA?9?$AA?5?$AAn?$AAo?$AAt?$AA?5?$AAe?$AAn?$AAo?$AAu?$AAg?$AAh?$AA?5?$AAs?$AAp?$AAa?$AAc?$AAe?$AA?5?$AAf?$AAo?$AAr?$AA?5?$AA_?$AAo@ 100037b8     LIBCMT:crt0msg.obj
 0001:00002828       ??_C@_1FC@ECHBIFBC@?$AAR?$AA6?$AA0?$AA1?$AA9?$AA?$AN?$AA?6?$AA?9?$AA?5?$AAu?$AAn?$AAa?$AAb?$AAl?$AAe?$AA?5?$AAt?$AAo?$AA?5?$AAo?$AAp?$AAe?$AAn?$AA?5?$AAc?$AAo?$AAn?$AAs?$AAo?$AAl?$AAe?$AA?5@ 10003828     LIBCMT:crt0msg.obj
 0001:00002880       ??_C@_1EC@JIBHAOPH@?$AAR?$AA6?$AA0?$AA1?$AA8?$AA?$AN?$AA?6?$AA?9?$AA?5?$AAu?$AAn?$AAe?$AAx?$AAp?$AAe?$AAc?$AAt?$AAe?$AAd?$AA?5?$AAh?$AAe?$AAa?$AAp?$AA?5?$AAe?$AAr?$AAr?$AAo?$AAr?$AA?$AN?$AA?6@ 10003880     LIBCMT:crt0msg.obj
 0001:000028c8       ??_C@_1FK@BEOGODMC@?$AAR?$AA6?$AA0?$AA1?$AA7?$AA?$AN?$AA?6?$AA?9?$AA?5?$AAu?$AAn?$AAe?$AAx?$AAp?$AAe?$AAc?$AAt?$AAe?$AAd?$AA?5?$AAm?$AAu?$AAl?$AAt?$AAi?$AAt?$AAh?$AAr?$AAe?$AAa?$AAd?$AA?5@ 100038c8     LIBCMT:crt0msg.obj
 0001:00002928       ??_C@_1FI@LOGNIKDM@?$AAR?$AA6?$AA0?$AA1?$AA6?$AA?$AN?$AA?6?$AA?9?$AA?5?$AAn?$AAo?$AAt?$AA?5?$AAe?$AAn?$AAo?$AAu?$AAg?$AAh?$AA?5?$AAs?$AAp?$AAa?$AAc?$AAe?$AA?5?$AAf?$AAo?$AAr?$AA?5?$AAt?$AAh@ 10003928     LIBCMT:crt0msg.obj
 0001:00002980       ??_C@_1EG@BEHAGFJD@?$AAR?$AA6?$AA0?$AA1?$AA0?$AA?$AN?$AA?6?$AA?9?$AA?5?$AAa?$AAb?$AAo?$AAr?$AAt?$AA?$CI?$AA?$CJ?$AA?5?$AAh?$AAa?$AAs?$AA?5?$AAb?$AAe?$AAe?$AAn?$AA?5?$AAc?$AAa?$AAl?$AAl?$AAe?$AAd@ 10003980     LIBCMT:crt0msg.obj
 0001:000029c8       ??_C@_1FI@HONFMGBI@?$AAR?$AA6?$AA0?$AA0?$AA9?$AA?$AN?$AA?6?$AA?9?$AA?5?$AAn?$AAo?$AAt?$AA?5?$AAe?$AAn?$AAo?$AAu?$AAg?$AAh?$AA?5?$AAs?$AAp?$AAa?$AAc?$AAe?$AA?5?$AAf?$AAo?$AAr?$AA?5?$AAe?$AAn@ 100039c8     LIBCMT:crt0msg.obj
 0001:00002a20       ??_C@_1FE@LLNEDJMD@?$AAR?$AA6?$AA0?$AA0?$AA8?$AA?$AN?$AA?6?$AA?9?$AA?5?$AAn?$AAo?$AAt?$AA?5?$AAe?$AAn?$AAo?$AAu?$AAg?$AAh?$AA?5?$AAs?$AAp?$AAa?$AAc?$AAe?$AA?5?$AAf?$AAo?$AAr?$AA?5?$AAa?$AAr@ 10003a20     LIBCMT:crt0msg.obj
 0001:00002a78       ??_C@_1FK@PGACCAFB@?$AAR?$AA6?$AA0?$AA0?$AA2?$AA?$AN?$AA?6?$AA?9?$AA?5?$AAf?$AAl?$AAo?$AAa?$AAt?$AAi?$AAn?$AAg?$AA?5?$AAp?$AAo?$AAi?$AAn?$AAt?$AA?5?$AAs?$AAu?$AAp?$AAp?$AAo?$AAr?$AAt?$AA?5@ 10003a78     LIBCMT:crt0msg.obj
 0001:00002b88       ??_C@_1EK@MBDPDCGA@?$AAM?$AAi?$AAc?$AAr?$AAo?$AAs?$AAo?$AAf?$AAt?$AA?5?$AAV?$AAi?$AAs?$AAu?$AAa?$AAl?$AA?5?$AAC?$AA?$CL?$AA?$CL?$AA?5?$AAR?$AAu?$AAn?$AAt?$AAi?$AAm?$AAe?$AA?5?$AAL?$AAi?$AAb@ 10003b88     LIBCMT:crt0msg.obj
 0001:00002bd4       ??_C@_15IABLJNFO@?$AA?6?$AA?6?$AA?$AA@ 10003bd4     LIBCMT:crt0msg.obj
 0001:00002bdc       ??_C@_17LGKOMLJ@?$AA?4?$AA?4?$AA?4?$AA?$AA@ 10003bdc     LIBCMT:crt0msg.obj
 0001:00002be4       ??_C@_1CO@EAEJAADC@?$AA?$DM?$AAp?$AAr?$AAo?$AAg?$AAr?$AAa?$AAm?$AA?5?$AAn?$AAa?$AAm?$AAe?$AA?5?$AAu?$AAn?$AAk?$AAn?$AAo?$AAw?$AAn?$AA?$DO?$AA?$AA@ 10003be4     LIBCMT:crt0msg.obj
 0001:00002c14       ??_C@_1DE@JNGNBFGO@?$AAR?$AAu?$AAn?$AAt?$AAi?$AAm?$AAe?$AA?5?$AAE?$AAr?$AAr?$AAo?$AAr?$AA?$CB?$AA?6?$AA?6?$AAP?$AAr?$AAo?$AAg?$AAr?$AAa?$AAm?$AA?3?$AA?5?$AA?$AA@ 10003c14     LIBCMT:crt0msg.obj
 0001:00002c4c       ??_7exception@std@@6B@     10003c4c     LIBCMT:stdexcpt.obj
 0001:00002c54       ??_C@_0BC@EOODALEL@Unknown?5exception?$AA@ 10003c54     LIBCMT:stdexcpt.obj
 0001:00002c6c       ??_7type_info@@6B@         10003c6c     LIBCMT:typinfo.obj
 0001:00002c90       ??_C@_05KLBDPFGC@e?$CL000?$AA@ 10003c90     LIBCMT:cvt.obj
 0001:00002c98       __XcptActTab               10003c98     LIBCMT:winxfltr.obj
 0001:00002d28       __First_FPE_Indx           10003d28     LIBCMT:winxfltr.obj
 0001:00002d2c       __Num_FPE                  10003d2c     LIBCMT:winxfltr.obj
 0001:00002d30       __XcptActTabSize           10003d30     LIBCMT:winxfltr.obj
 0001:00002d34       __XcptActTabCount          10003d34     LIBCMT:winxfltr.obj
 0001:00002d38       ___newctype                10003d38     LIBCMT:ctype.obj
 0001:00003038       __wctype                   10004038     LIBCMT:ctype.obj
 0001:00003240       ___newclmap                10004240     LIBCMT:ctype.obj
 0001:000033c0       ___newcumap                100043c0     LIBCMT:ctype.obj
 0001:00003540       ??_C@_0BI@DFKBFLJE@GetProcessWindowStation?$AA@ 10004540     LIBCMT:crtmboxw.obj
 0001:00003558       ??_C@_0BK@DEKFELLI@GetUserObjectInformationW?$AA@ 10004558     LIBCMT:crtmboxw.obj
 0001:00003574       ??_C@_0BD@HHGDFDBJ@GetLastActivePopup?$AA@ 10004574     LIBCMT:crtmboxw.obj
 0001:00003588       ??_C@_0BA@HNOPNCHB@GetActiveWindow?$AA@ 10004588     LIBCMT:crtmboxw.obj
 0001:00003598       ??_C@_0M@DLDCCGNP@MessageBoxW?$AA@ 10004598     LIBCMT:crtmboxw.obj
 0001:000035a4       ??_C@_1BG@GOEBHBDC@?$AAU?$AAS?$AAE?$AAR?$AA3?$AA2?$AA?4?$AAD?$AAL?$AAL?$AA?$AA@ 100045a4     LIBCMT:crtmboxw.obj
 0001:000035c4       ??_C@_0BK@CFCOFLF@?5Complete?5Object?5Locator?8?$AA@ 100045c4     LIBCMT:undname.obj
 0001:000035e0       ??_C@_0BN@MECKDCOJ@?5Class?5Hierarchy?5Descriptor?8?$AA@ 100045e0     LIBCMT:undname.obj
 0001:00003600       ??_C@_0BD@LGICGFMM@?5Base?5Class?5Array?8?$AA@ 10004600     LIBCMT:undname.obj
 0001:00003614       ??_C@_0BM@LDKODKLH@?5Base?5Class?5Descriptor?5at?5?$CI?$AA@ 10004614     LIBCMT:undname.obj
 0001:00003630       ??_C@_0BC@DAFEJGAK@?5Type?5Descriptor?8?$AA@ 10004630     LIBCMT:undname.obj
 0001:00003644       ??_C@_0BM@PMGGMLDN@?$GAlocal?5static?5thread?5guard?8?$AA@ 10004644     LIBCMT:undname.obj
 0001:00003660       ??_C@_0CL@FGIJHLCE@?$GAmanaged?5vector?5copy?5constructor@ 10004660     LIBCMT:undname.obj
 0001:0000368c       ??_C@_0CJ@GJELGAMM@?$GAvector?5vbase?5copy?5constructor?5i@ 1000468c     LIBCMT:undname.obj
 0001:000036b8       ??_C@_0CD@CGAJBKEJ@?$GAvector?5copy?5constructor?5iterato@ 100046b8     LIBCMT:undname.obj
 0001:000036dc       ??_C@_0CB@PDBIFEP@?$GAdynamic?5atexit?5destructor?5for?5?8@ 100046dc     LIBCMT:undname.obj
 0001:00003700       ??_C@_0BL@CLIPGLGB@?$GAdynamic?5initializer?5for?5?8?$AA@ 10004700     LIBCMT:undname.obj
 0001:0000371c       ??_C@_0CM@FCBBDIGB@?$GAeh?5vector?5vbase?5copy?5constructo@ 1000471c     LIBCMT:undname.obj
 0001:00003748       ??_C@_0CG@HLDDJMAG@?$GAeh?5vector?5copy?5constructor?5iter@ 10004748     LIBCMT:undname.obj
 0001:00003770       ??_C@_0CF@IMGKMJNO@?$GAmanaged?5vector?5destructor?5itera@ 10004770     LIBCMT:undname.obj
 0001:00003798       ??_C@_0CG@CFDHKGGD@?$GAmanaged?5vector?5constructor?5iter@ 10004798     LIBCMT:undname.obj
 0001:000037c0       ??_C@_0BN@CKNJLHMB@?$GAplacement?5delete?$FL?$FN?5closure?8?$AA@ 100047c0     LIBCMT:undname.obj
 0001:000037e0       ??_C@_0BL@CNOONJFP@?$GAplacement?5delete?5closure?8?$AA@ 100047e0     LIBCMT:undname.obj
 0001:000037fc       ??_C@_0P@HJKNJFNN@?$GAomni?5callsig?8?$AA@ 100047fc     LIBCMT:undname.obj
 0001:0000380c       ??_C@_09LBNFPBCA@?5delete?$FL?$FN?$AA@ 1000480c     LIBCMT:undname.obj
 0001:00003818       ??_C@_06FHBGPFGH@?5new?$FL?$FN?$AA@ 10004818     LIBCMT:undname.obj
 0001:00003820       ??_C@_0CE@IIHCMGGL@?$GAlocal?5vftable?5constructor?5closu@ 10004820     LIBCMT:undname.obj
 0001:00003844       ??_C@_0BA@KKLDJDLB@?$GAlocal?5vftable?8?$AA@ 10004844     LIBCMT:undname.obj
 0001:00003854       ??_C@_05KHLCHHI@?$GARTTI?$AA@ 10004854     LIBCMT:undname.obj
 0001:0000385c       ??_C@_03KLGMFNMG@?$GAEH?$AA@ 1000485c     LIBCMT:undname.obj
 0001:00003860       ??_C@_0BA@KBCDOMBN@?$GAudt?5returning?8?$AA@ 10004860     LIBCMT:undname.obj
 0001:00003870       ??_C@_0BL@LLKPOHJI@?$GAcopy?5constructor?5closure?8?$AA@ 10004870     LIBCMT:undname.obj
 0001:0000388c       ??_C@_0CH@OOJPLCPH@?$GAeh?5vector?5vbase?5constructor?5ite@ 1000488c     LIBCMT:undname.obj
 0001:000038b4       ??_C@_0CA@GCEOPDGL@?$GAeh?5vector?5destructor?5iterator?8?$AA@ 100048b4     LIBCMT:undname.obj
 0001:000038d4       ??_C@_0CB@JONCMFFK@?$GAeh?5vector?5constructor?5iterator?8@ 100048d4     LIBCMT:undname.obj
 0001:000038f8       ??_C@_0BL@NILFHHPC@?$GAvirtual?5displacement?5map?8?$AA@ 100048f8     LIBCMT:undname.obj
 0001:00003914       ??_C@_0CE@IKBNEHA@?$GAvector?5vbase?5constructor?5iterat@ 10004914     LIBCMT:undname.obj
 0001:00003938       ??_C@_0BN@LFPFMEDL@?$GAvector?5destructor?5iterator?8?$AA@ 10004938     LIBCMT:undname.obj
 0001:00003958       ??_C@_0BO@PFGOCPJJ@?$GAvector?5constructor?5iterator?8?$AA@ 10004958     LIBCMT:undname.obj
 0001:00003978       ??_C@_0BN@IMDCHIKM@?$GAscalar?5deleting?5destructor?8?$AA@ 10004978     LIBCMT:undname.obj
 0001:00003998       ??_C@_0BO@OBMKPJIG@?$GAdefault?5constructor?5closure?8?$AA@ 10004998     LIBCMT:undname.obj
 0001:000039b8       ??_C@_0BN@DEGPLNFK@?$GAvector?5deleting?5destructor?8?$AA@ 100049b8     LIBCMT:undname.obj
 0001:000039d8       ??_C@_0BD@JDLKDPAB@?$GAvbase?5destructor?8?$AA@ 100049d8     LIBCMT:undname.obj
 0001:000039ec       ??_C@_08OBABFOLI@?$GAstring?8?$AA@ 100049ec     LIBCMT:undname.obj
 0001:000039f8       ??_C@_0BF@KDPPACIK@?$GAlocal?5static?5guard?8?$AA@ 100049f8     LIBCMT:undname.obj
 0001:00003a10       ??_C@_08LLFFHHDJ@?$GAtypeof?8?$AA@ 10004a10     LIBCMT:undname.obj
 0001:00003a1c       ??_C@_07FEEIOKP@?$GAvcall?8?$AA@ 10004a1c     LIBCMT:undname.obj
 0001:00003a24       ??_C@_09BLBHBJP@?$GAvbtable?8?$AA@ 10004a24     LIBCMT:undname.obj
 0001:00003a30       ??_C@_09IFPLHPGF@?$GAvftable?8?$AA@ 10004a30     LIBCMT:undname.obj
 0001:00003a3c       ??_C@_02MHEGNOJ@?$FO?$DN?$AA@ 10004a3c     LIBCMT:undname.obj
 0001:00003a40       ??_C@_02DHLNPPGH@?$HM?$DN?$AA@ 10004a40     LIBCMT:undname.obj
 0001:00003a44       ??_C@_02FGJGFEAB@?$CG?$DN?$AA@ 10004a44     LIBCMT:undname.obj
 0001:00003a48       ??_C@_03CDNPDDLA@?$DM?$DM?$DN?$AA@ 10004a48     LIBCMT:undname.obj
 0001:00003a4c       ??_C@_03IKFCCPFF@?$DO?$DO?$DN?$AA@ 10004a4c     LIBCMT:undname.obj
 0001:00003a50       ??_C@_02FENAOKFI@?$CF?$DN?$AA@ 10004a50     LIBCMT:undname.obj
 0001:00003a54       ??_C@_02FJEHGPIO@?1?$DN?$AA@ 10004a54     LIBCMT:undname.obj
 0001:00003a58       ??_C@_02FKMDLLOA@?9?$DN?$AA@ 10004a58     LIBCMT:undname.obj
 0001:00003a5c       ??_C@_02FOEOMHFC@?$CL?$DN?$AA@ 10004a5c     LIBCMT:undname.obj
 0001:00003a60       ??_C@_02FPIMKNGF@?$CK?$DN?$AA@ 10004a60     LIBCMT:undname.obj
 0001:00003a64       ??_C@_02NONPIBCD@?$HM?$HM?$AA@ 10004a64     LIBCMT:undname.obj
 0001:00003a68       ??_C@_02PPKAJPJL@?$CG?$CG?$AA@ 10004a68     LIBCMT:undname.obj
 0001:00003a6c       ??_C@_01DNKMNLPK@?$HM?$AA@ 10004a6c     LIBCMT:undname.obj
 0001:00003a70       ??_C@_01JKBOJNNK@?$FO?$AA@ 10004a70     LIBCMT:undname.obj
 0001:00003a74       ??_C@_01PJKLJHI@?$HO?$AA@  10004a74     LIBCMT:undname.obj
 0001:00003a78       ??_C@_02HCKGKOFO@?$CI?$CJ?$AA@ 10004a78     LIBCMT:undname.obj
 0001:00003a7c       ??_C@_01IHBHIGKO@?0?$AA@   10004a7c     LIBCMT:undname.obj
 0001:00003a80       ??_C@_02EEKDKGMJ@?$DO?$DN?$AA@ 10004a80     LIBCMT:undname.obj
 0001:00003a84       ??_C@_01PPODPGHN@?$DO?$AA@ 10004a84     LIBCMT:undname.obj
 0001:00003a88       ??_C@_02EHCHHCKH@?$DM?$DN?$AA@ 10004a88     LIBCMT:undname.obj
 0001:00003a8c       ??_C@_01MNNFJEPP@?$DM?$AA@ 10004a8c     LIBCMT:undname.obj
 0001:00003a90       ??_C@_01FGNFDNOH@?$CF?$AA@ 10004a90     LIBCMT:undname.obj
 0001:00003a94       ??_C@_01KMDKNFGN@?1?$AA@   10004a94     LIBCMT:undname.obj
 0001:00003a98       ??_C@_03MNHNFDLC@?9?$DO?$CK?$AA@ 10004a98     LIBCMT:undname.obj
 0001:00003a9c       ??_C@_01HNPIGOCE@?$CG?$AA@ 10004a9c     LIBCMT:undname.obj
 0001:00003aa0       ??_C@_01MIFGBAGJ@?$CL?$AA@ 10004aa0     LIBCMT:undname.obj
 0001:00003aa4       ??_C@_01JOAMLHOP@?9?$AA@   10004aa4     LIBCMT:undname.obj
 0001:00003aa8       ??_C@_02BAABKJLB@?9?9?$AA@ 10004aa8     LIBCMT:undname.obj
 0001:00003aac       ??_C@_02ECNGHCIF@?$CL?$CL?$AA@ 10004aac     LIBCMT:undname.obj
 0001:00003ab0       ??_C@_01NBENCBCI@?$CK?$AA@ 10004ab0     LIBCMT:undname.obj
 0001:00003ab4       ??_C@_02HBOOOICD@?9?$DO?$AA@ 10004ab4     LIBCMT:undname.obj
 0001:00003ab8       ??_C@_08LHJFAFGD@operator?$AA@ 10004ab8     LIBCMT:undname.obj
 0001:00003ac4       ??_C@_02GPECMEKF@?$FL?$FN?$AA@ 10004ac4     LIBCMT:undname.obj
 0001:00003ac8       ??_C@_02FDNJECIE@?$CB?$DN?$AA@ 10004ac8     LIBCMT:undname.obj
 0001:00003acc       ??_C@_02EGOFBIJA@?$DN?$DN?$AA@ 10004acc     LIBCMT:undname.obj
 0001:00003ad0       ??_C@_01DCLJPIOD@?$CB?$AA@ 10004ad0     LIBCMT:undname.obj
 0001:00003ad4       ??_C@_02FODMEDOG@?$DM?$DM?$AA@ 10004ad4     LIBCMT:undname.obj
 0001:00003ad8       ??_C@_02GPIOPFAK@?$DO?$DO?$AA@ 10004ad8     LIBCMT:undname.obj
 0001:00003adc       ??_C@_07FPCDHGMM@?5delete?$AA@ 10004adc     LIBCMT:undname.obj
 0001:00003ae4       ??_C@_04NIHEBCM@?5new?$AA@ 10004ae4     LIBCMT:undname.obj
 0001:00003aec       ??_C@_0M@GFIIJFMG@__unaligned?$AA@ 10004aec     LIBCMT:undname.obj
 0001:00003af8       ??_C@_0L@PILCLIHE@__restrict?$AA@ 10004af8     LIBCMT:undname.obj
 0001:00003b04       ??_C@_07JOMMBBKO@__ptr64?$AA@ 10004b04     LIBCMT:undname.obj
 0001:00003b0c       ??_C@_06GHPCKEAG@__eabi?$AA@ 10004b0c     LIBCMT:undname.obj
 0001:00003b14       ??_C@_09HIJEGCPM@__clrcall?$AA@ 10004b14     LIBCMT:undname.obj
 0001:00003b20       ??_C@_0L@JMKHOMEK@__fastcall?$AA@ 10004b20     LIBCMT:undname.obj
 0001:00003b2c       ??_C@_0L@NPHFGOKO@__thiscall?$AA@ 10004b2c     LIBCMT:undname.obj
 0001:00003b38       ??_C@_09IFJBGAPI@__stdcall?$AA@ 10004b38     LIBCMT:undname.obj
 0001:00003b44       ??_C@_08GHMPAG@__pascal?$AA@ 10004b44     LIBCMT:undname.obj
 0001:00003b50       ??_C@_07KOLFKCDI@__cdecl?$AA@ 10004b50     LIBCMT:undname.obj
 0001:00003b58       ??_C@_08EHJDFFNH@__based?$CI?$AA@ 10004b58     LIBCMT:undname.obj
 0001:00003cec       ??_C@_06IMKFLFPG@1?$CDQNAN?$AA@ 10004cec     LIBCMT:_x10fout_.obj
 0001:00003cf4       ??_C@_05DNEBIAHO@1?$CDINF?$AA@ 10004cf4     LIBCMT:_x10fout_.obj
 0001:00003cfc       ??_C@_05PHHOCPM@1?$CDIND?$AA@ 10004cfc     LIBCMT:_x10fout_.obj
 0001:00003d04       ??_C@_06PGGFOGJG@1?$CDSNAN?$AA@ 10004d04     LIBCMT:_x10fout_.obj
 0001:00003d10       __load_config_used         10004d10     LIBCMT:loadcfg.obj
 0001:00003d58       ??_R4bad_alloc@std@@6B@    10004d58     LIBCMT:new.obj
 0001:00003d6c       ??_R3bad_alloc@std@@8      10004d6c     LIBCMT:new.obj
 0001:00003d7c       ??_R2bad_alloc@std@@8      10004d7c     LIBCMT:new.obj
 0001:00003d88       ??_R1A@?0A@EA@bad_alloc@std@@8 10004d88     LIBCMT:new.obj
 0001:00003da4       ??_R1A@?0A@EA@exception@std@@8 10004da4     LIBCMT:new.obj
 0001:00003dc0       ??_R3exception@std@@8      10004dc0     LIBCMT:new.obj
 0001:00003dd0       ??_R2exception@std@@8      10004dd0     LIBCMT:new.obj
 0001:00003dd8       ??_R4exception@std@@6B@    10004dd8     LIBCMT:stdexcpt.obj
 0001:00003dec       ??_R4type_info@@6B@        10004dec     LIBCMT:typinfo.obj
 0001:00003e00       ??_R3type_info@@8          10004e00     LIBCMT:typinfo.obj
 0001:00003e10       ??_R2type_info@@8          10004e10     LIBCMT:typinfo.obj
 0001:00003e18       ??_R1A@?0A@EA@type_info@@8 10004e18     LIBCMT:typinfo.obj
 0001:00003e40       ___safe_se_handler_table   10004e40     <linker-defined>
 0001:00003e4c       ___rtc_iaa                 10004e4c     LIBCMT:_initsect_.obj
 0001:00003e50       ___rtc_izz                 10004e50     LIBCMT:_initsect_.obj
 0001:00003e54       ___rtc_taa                 10004e54     LIBCMT:_initsect_.obj
 0001:00003e58       ___rtc_tzz                 10004e58     LIBCMT:_initsect_.obj
 0001:00003e60       __chkstk                   10004e60 f   chkstk.obj
 0001:00003e60       __alloca_probe             10004e60     chkstk.obj
 0001:00003e90       ?fputc@@YAHHPAX@Z          10004e90 f   fileio.obj
 0001:00004790       ?PrintHandleInfo@@YA_NKPAX_NPAVPerfThread@@@Z 10005790 f   handles.obj
 0001:00004930       ?GetLangString@PluginDialogBuilder@@MAEPB_WH@Z 10005930 f i PCFG.OBJ
 0001:00004950       ?Write@_Opt@@SAXXZ         10005950 f   PCFG.OBJ
 0001:00004ba0       ?Read@_Opt@@SAXXZ          10005ba0 f   PCFG.OBJ
 0001:00004ed0       ?InitDialogItem@?$DialogBuilderBase@UFarDialogItem@@@@MAEXPAUFarDialogItem@@PB_W@Z 10005ed0 f i PCFG.OBJ
 0001:00004ed0       ?SaveValue@?$DialogItemBinding@UFarDialogItem@@@@UAEXPAUFarDialogItem@@H@Z 10005ed0 f i PCFG.OBJ
 0001:00004ee0       ?TextWidth@?$DialogBuilderBase@UFarDialogItem@@@@MAEHABUFarDialogItem@@@Z 10005ee0 f i PCFG.OBJ
 0001:00004ef0       ?GetLangString@?$DialogBuilderBase@UFarDialogItem@@@@MAEPB_WH@Z 10005ef0 f i PCFG.OBJ
 0001:00004ef0       ?CreateRadioButtonBinding@?$DialogBuilderBase@UFarDialogItem@@@@MAEPAU?$DialogItemBinding@UFarDialogItem@@@@PAH@Z 10005ef0 f i PCFG.OBJ
 0001:00004f00       ?DoShowDialog@?$DialogBuilderBase@UFarDialogItem@@@@MAEHXZ 10005f00 f i PCFG.OBJ
 0001:00004f10       ?CreateCheckBoxBinding@?$DialogBuilderBase@UFarDialogItem@@@@MAEPAU?$DialogItemBinding@UFarDialogItem@@@@PAHH@Z 10005f10 f i PCFG.OBJ
 0001:00004f10       ?AddUIntEditField@?$DialogBuilderBase@UFarDialogItem@@@@UAEPAUFarDialogItem@@PAIH@Z 10005f10 f i PCFG.OBJ
 0001:00004f10       ?AddIntEditField@?$DialogBuilderBase@UFarDialogItem@@@@UAEPAUFarDialogItem@@PAHH@Z 10005f10 f i PCFG.OBJ
 0001:00004f20       ??1?$DialogBuilderBase@UFarDialogItem@@@@MAE@XZ 10005f20 f i PCFG.OBJ
 0001:00004f70       ??_G?$DialogBuilderBase@UFarDialogItem@@@@MAEPAXI@Z 10005f70 f i PCFG.OBJ
 0001:00004f70       ??_E?$DialogBuilderBase@UFarDialogItem@@@@MAEPAXI@Z 10005f70 f i PCFG.OBJ
 0001:00004f90       ?ReallocDialogItems@?$DialogBuilderBase@UFarDialogItem@@@@IAEXXZ 10005f90 f i PCFG.OBJ
 0001:00005060       ?UpdateSecondColumnPosition@?$DialogBuilderBase@UFarDialogItem@@@@IAEXXZ 10006060 f i PCFG.OBJ
 0001:000050c0       ?SaveValues@?$DialogBuilderBase@UFarDialogItem@@@@IAEXXZ 100060c0 f i PCFG.OBJ
 0001:00005110       ?MaxTextWidth@?$DialogBuilderBase@UFarDialogItem@@@@IAEHXZ 10006110 f i PCFG.OBJ
 0001:000051d0       ??1PluginDialogBuilder@@UAE@XZ 100061d0 f i PCFG.OBJ
 0001:000051f0       ?InitDialogItem@PluginDialogBuilder@@MAEXPAUFarDialogItem@@PB_W@Z 100061f0 f i PCFG.OBJ
 0001:00005210       ?TextWidth@PluginDialogBuilder@@MAEHABUFarDialogItem@@@Z 10006210 f i PCFG.OBJ
 0001:00005230       ?DoShowDialog@PluginDialogBuilder@@MAEHXZ 10006230 f i PCFG.OBJ
 0001:00005290       ??_EPluginRadioButtonBinding@@UAEPAXI@Z 10006290 f i PCFG.OBJ
 0001:00005290       ??_GPluginEditFieldBinding@@UAEPAXI@Z 10006290 f i Pclass.obj
 0001:00005290       ??_G?$DialogItemBinding@UFarDialogItem@@@@UAEPAXI@Z 10006290 f i PCFG.OBJ
 0001:00005290       ??_GPluginCheckBoxBinding@@UAEPAXI@Z 10006290 f i PCFG.OBJ
 0001:00005290       ??_EPluginEditFieldBinding@@UAEPAXI@Z 10006290 f i Pclass.obj
 0001:00005290       ??_GPluginIntEditFieldBinding@@UAEPAXI@Z 10006290 f i PCFG.OBJ
 0001:00005290       ??_GPluginRadioButtonBinding@@UAEPAXI@Z 10006290 f i PCFG.OBJ
 0001:00005290       ??_EPluginIntEditFieldBinding@@UAEPAXI@Z 10006290 f i PCFG.OBJ
 0001:00005290       ??_EPluginCheckBoxBinding@@UAEPAXI@Z 10006290 f i PCFG.OBJ
 0001:00005290       ??_E?$DialogItemBinding@UFarDialogItem@@@@UAEPAXI@Z 10006290 f i PCFG.OBJ
 0001:00005290       ??_EPluginUIntEditFieldBinding@@UAEPAXI@Z 10006290 f i PCFG.OBJ
 0001:00005290       ??_GPluginUIntEditFieldBinding@@UAEPAXI@Z 10006290 f i PCFG.OBJ
 0001:000052b0       ?SaveValue@PluginCheckBoxBinding@@UAEXPAUFarDialogItem@@H@Z 100062b0 f i PCFG.OBJ
 0001:000052f0       ?SaveValue@PluginRadioButtonBinding@@UAEXPAUFarDialogItem@@H@Z 100062f0 f i PCFG.OBJ
 0001:00005320       ??0PluginIntEditFieldBinding@@QAE@ABUPluginStartupInfo@@PAPAXHPAHH@Z 10006320 f i PCFG.OBJ
 0001:000053c0       ?SaveValue@PluginIntEditFieldBinding@@UAEXPAUFarDialogItem@@H@Z 100063c0 f i PCFG.OBJ
 0001:000053f0       ??0PluginUIntEditFieldBinding@@QAE@ABUPluginStartupInfo@@PAPAXHPAIH@Z 100063f0 f i PCFG.OBJ
 0001:00005490       ?SaveValue@PluginUIntEditFieldBinding@@UAEXPAUFarDialogItem@@H@Z 10006490 f i PCFG.OBJ
 0001:000054c0       ?CreateCheckBoxBinding@PluginDialogBuilder@@MAEPAU?$DialogItemBinding@UFarDialogItem@@@@PAHH@Z 100064c0 f i PCFG.OBJ
 0001:00005510       ?CreateRadioButtonBinding@PluginDialogBuilder@@MAEPAU?$DialogItemBinding@UFarDialogItem@@@@PAH@Z 10006510 f i PCFG.OBJ
 0001:00005560       ??_GPluginDialogBuilder@@UAEPAXI@Z 10006560 f i PCFG.OBJ
 0001:00005560       ??_EPluginDialogBuilder@@UAEPAXI@Z 10006560 f i PCFG.OBJ
 0001:000055a0       ?AddText@?$DialogBuilderBase@UFarDialogItem@@@@QAEPAUFarDialogItem@@H@Z 100065a0 f i PCFG.OBJ
 0001:00005620       ?AddCheckbox@?$DialogBuilderBase@UFarDialogItem@@@@QAEPAUFarDialogItem@@HPAHH_N@Z 10006620 f i PCFG.OBJ
 0001:00005750       ?AddSeparator@?$DialogBuilderBase@UFarDialogItem@@@@QAEXPB_W@Z 10006750 f i PCFG.OBJ
 0001:000057c0       ?AddButtons@?$DialogBuilderBase@UFarDialogItem@@@@QAEXHPBHHH@Z 100067c0 f i PCFG.OBJ
 0001:00005920       ?UpdateBorderSize@?$DialogBuilderBase@UFarDialogItem@@@@IAEXXZ 10006920 f i PCFG.OBJ
 0001:000059c0       ??0PluginDialogBuilder@@QAE@ABUPluginStartupInfo@@ABU_GUID@@1HPB_WP6GHPAXHH3@Z3_K@Z 100069c0 f i PCFG.OBJ
 0001:00005ad0       ?AddIntEditField@PluginDialogBuilder@@UAEPAUFarDialogItem@@PAHH@Z 10006ad0 f i PCFG.OBJ
 0001:00005b90       ?AddUIntEditField@PluginDialogBuilder@@UAEPAUFarDialogItem@@PAIH@Z 10006b90 f i PCFG.OBJ
 0001:00005c50       ?ShowDialog@?$DialogBuilderBase@UFarDialogItem@@@@QAE_NXZ 10006c50 f i PCFG.OBJ
 0001:00005c90       ?Config@@YAHXZ             10006c90 f   PCFG.OBJ
 0001:00005ed0       ??0ui64Table@@QAE@XZ       10006ed0 f   Pclass.obj
 0001:00005fc0       ?SavePanelModes@Plist@@SAXXZ 10006fc0 f   Pclass.obj
 0001:00006210       ?TranslateMode@Plist@@CA_NPB_WPA_W@Z 10007210 f   Pclass.obj
 0001:00006420       ?GeneratePanelModes@Plist@@AAEXXZ 10007420 f   Pclass.obj
 0001:000069d0       ?PanelModes@Plist@@QAEPAUPanelMode@@AAI@Z 100079d0 f   Pclass.obj
 0001:00006a60       ?GetOpenPanelInfo@Plist@@QAEXPAUOpenPanelInfo@@@Z 10007a60 f   Pclass.obj
 0001:00006b60       ?EnumWndProc@@YGHPAUHWND__@@J@Z 10007b60 f   Pclass.obj
 0001:00006be0       ?FreeFindData@Plist@@QAEXPAUPluginPanelItem@@H@Z 10007be0 f   Pclass.obj
 0001:00006c40       ?Reread@Plist@@AAEXXZ      10007c40 f   Pclass.obj
 0001:00006cc0       ?PutToCmdLine@Plist@@AAEXPA_W@Z 10007cc0 f   Pclass.obj
 0001:00006d70       ?PrintTitle@Plist@@SAPA_WH@Z 10007d70 f   Pclass.obj
 0001:00006dc0       ?FileTimeToText@Plist@@AAEXPAU_FILETIME@@0PA_W@Z 10007dc0 f   Pclass.obj
 0001:00006f00       ?GetVersionInfo@Plist@@SA_NPA_WAAPAEAAPA_W2@Z 10007f00 f   Pclass.obj
 0001:00007050       ?PrintVersionInfo@Plist@@AAEXPAXPA_W@Z 10008050 f   Pclass.obj
 0001:00007120       ?ConnectWMI@Plist@@AAE_NXZ 10008120 f   Pclass.obj
 0001:000071a0       ?PrintOwnerInfo@Plist@@AAEXPAXK@Z 100081a0 f   Pclass.obj
 0001:00007390       ?Compare@Plist@@QAEHPBUPluginPanelItem@@0I@Z 10008390 f   Pclass.obj
 0001:00007540       ?WmiError@Plist@@AAEXXZ    10008540 f   Pclass.obj
 0001:00007580       ??0?$Array@_W@@QAE@K@Z     10008580 f i Pclass.obj
 0001:000075c0       ??0?$Array@UFarMenuItem@@@@QAE@K@Z 100085c0 f i Pclass.obj
 0001:00007600       ?SaveValue@PluginEditFieldBinding@@UAEXPAUFarDialogItem@@H@Z 10008600 f i Pclass.obj
 0001:00007630       ?InitializePanelModes@Plist@@SAXXZ 10008630 f   Pclass.obj
 0001:00007a80       ?GetFindData@Plist@@QAEHAAPAUPluginPanelItem@@AAI_K@Z 10008a80 f   Pclass.obj
 0001:00008180       ?GetFiles@Plist@@QAEHPAUPluginPanelItem@@HHPAPB_W_KAAU_Opt@@@Z 10009180 f   Pclass.obj
 0001:00008ee0       ?DeleteFiles@Plist@@QAEHPAUPluginPanelItem@@H_K@Z 10009ee0 f   Pclass.obj
 0001:000091c0       ?ProcessEvent@Plist@@QAEHHPAX@Z 1000a1c0 f   Pclass.obj
 0001:00009380       ?DisconnectWMI@Plist@@AAEXXZ 1000a380 f   Pclass.obj
 0001:000093b0       ?EndColumns@?$DialogBuilderBase@UFarDialogItem@@@@QAEXXZ 1000a3b0 f i Pclass.obj
 0001:00009470       ?AddEditField@PluginDialogBuilder@@QAEPAUFarDialogItem@@PA_WHHPB_W_N@Z 1000a470 f i Pclass.obj
 0001:00009570       ?AddPasswordField@PluginDialogBuilder@@QAEPAUFarDialogItem@@PA_WHH@Z 1000a570 f i Pclass.obj
 0001:00009640       ??0Plist@@QAE@XZ           1000a640 f   Pclass.obj
 0001:000097c0       ??1Plist@@QAE@XZ           1000a7c0 f   Pclass.obj
 0001:00009810       ?Connect@Plist@@QAE_NPB_W00@Z 1000a810 f   Pclass.obj
 0001:00009a00       ?ProcessKey@Plist@@QAEHPBU_INPUT_RECORD@@@Z 1000aa00 f   Pclass.obj
 0001:0000a980       ?SyncReread@PerfThread@@QAEXXZ 1000b980 f   perfthread.obj
 0001:0000a9b0       ?GetProcessData@PerfThread@@QBEPAUProcessPerfData@@KK@Z 1000b9b0 f   perfthread.obj
 0001:0000aa10       ?Refresh@PerfThread@@AAEXXZ 1000ba10 f   perfthread.obj
 0001:0000b290       ?RefreshWMIData@PerfThread@@AAEXXZ 1000c290 f   perfthread.obj
 0001:0000b3b0       ?ThreadProc@PerfThread@@AAGKXZ 1000c3b0 f   perfthread.obj
 0001:0000b470       ?ThreadProc@PerfThread@@CGKPAX@Z 1000c470 f   perfthread.obj
 0001:0000b480       ??0PerfThread@@QAE@AAVPlist@@PB_W11@Z 1000c480 f   perfthread.obj
 0001:0000b850       ??1PerfThread@@QAE@XZ      1000c850 f   perfthread.obj
 0001:0000b8d0       ?GetInternalProcessData@@YAHPAXPAU_LDR_MODULE@@AAPAU_RTL_USER_PROCESS_PARAMETERS@@AAPAD_N@Z 1000c8d0 f   Plist.obj
 0001:0000b9c0       ?GetPDataNT@@YA_NAAUProcessDataNT@@AAUProcessPerfData@@@Z 1000c9c0 f   Plist.obj
 0001:0000ba50       ?Enable@DebugToken@@QAE_NXZ 1000ca50 f   Plist.obj
 0001:0000bac0       ?Revert@DebugToken@@QAE_NXZ 1000cac0 f   Plist.obj
 0001:0000bb00       ?CreateToken@DebugToken@@SA_NXZ 1000cb00 f   Plist.obj
 0001:0000bbe0       ?PrintTime@@YAPA_WK_N@Z    1000cbe0 f   Plist.obj
 0001:0000bc70       ?PrintTime@@YAPA_W_K_N@Z   1000cc70 f   Plist.obj
 0001:0000bce0       ?DumpNTCounters@@YAXPAXAAVPerfThread@@KK@Z 1000cce0 f   Plist.obj
 0001:0000bf80       ?PrintModuleVersion@@YAXPAXPA_W1H@Z 1000cf80 f   Plist.obj
 0001:0000c050       ?OpenProcessForced@@YAPAXPAVDebugToken@@KKH@Z 1000d050 f   Plist.obj
 0001:0000c0a0       ?GetList@@YAHAAPAUPluginPanelItem@@AAIAAVPerfThread@@@Z 1000d0a0 f   Plist.obj
 0001:0000c350       ?GetOpenProcessData@@YAXPAXPA_WK1K1KPAPA_W2@Z 1000d350 f   Plist.obj
 0001:0000c630       ?KillProcess@@YAHKPAUHWND__@@@Z 1000d630 f   Plist.obj
 0001:0000c720       ?PrintNTCurDirAndEnv@@YAXPAX0H@Z 1000d720 f   Plist.obj
 0001:0000c860       ?PrintModules@@YAXPAXKAAU_Opt@@@Z 1000d860 f   Plist.obj
 0001:0000ca70       ?GetMsg@@YAPB_WH@Z         1000da70 f   Pmix.obj
 0001:0000ca90       ?ConvertDate@@YAXABU_FILETIME@@PA_W1@Z 1000da90 f   Pmix.obj
 0001:0000cb20       ?WinError@@YAHPA_W@Z       1000db20 f   Pmix.obj
 0001:0000cc80       ??0WMIConnection@@QAE@XZ   1000dc80 f   WMI.obj
 0001:0000cca0       ?GetProcessExecutablePath@WMIConnection@@QAEXKPA_W@Z 1000dca0 f   WMI.obj
 0001:0000cd70       ?GetProcessPriority@WMIConnection@@QAEKK@Z 1000dd70 f   WMI.obj
 0001:0000ce30       ?GetProcessOwner@WMIConnection@@QAEXKPA_W0@Z 1000de30 f   WMI.obj
 0001:0000cf90       ?GetProcessUserSid@WMIConnection@@QAEXKPA_W@Z 1000df90 f   WMI.obj
 0001:0000d080       ?GetProcessSessionId@WMIConnection@@QAEHK@Z 1000e080 f   WMI.obj
 0001:0000d140       ?ExecMethod@WMIConnection@@AAEHKPB_W0K@Z 1000e140 f   WMI.obj
 0001:0000d350       ?SetProcessPriority@WMIConnection@@QAEHKK@Z 1000e350 f   WMI.obj
 0001:0000d370       ?TerminateProcess@WMIConnection@@QAEHK@Z 1000e370 f   WMI.obj
 0001:0000d390       ?Connect@WMIConnection@@QAE_NPB_W00@Z 1000e390 f   WMI.obj
 0001:0000d4f0       ?Disconnect@WMIConnection@@QAEXXZ 1000e4f0 f   WMI.obj
 0001:0000d510       ??1WMIConnection@@QAE@XZ   1000e510 f   WMI.obj
 0001:0000d6d0       ?Message@@YAHIPA_WPAPB_WHH@Z 1000e6d0 f   Proclist.obj
 0001:0000d700       _GetGlobalInfoW@4          1000e700 f   Proclist.obj
 0001:0000d780       _SetStartupInfoW@4         1000e780 f   Proclist.obj
 0001:0000d800       _ExitFARW@4                1000e800 f   Proclist.obj
 0001:0000d820       _ClosePanelW@4             1000e820 f   Proclist.obj
 0001:0000d840       _GetFindDataW@4            1000e840 f   Proclist.obj
 0001:0000d860       _FreeFindDataW@4           1000e860 f   Proclist.obj
 0001:0000d880       _GetPluginInfoW@4          1000e880 f   Proclist.obj
 0001:0000d930       _GetOpenPanelInfoW@4       1000e930 f   Proclist.obj
 0001:0000d940       _GetFilesW@4               1000e940 f   Proclist.obj
 0001:0000d970       _DeleteFilesW@4            1000e970 f   Proclist.obj
 0001:0000d990       _ProcessPanelEventW@4      1000e990 f   Proclist.obj
 0001:0000d9b0       _ProcessPanelInputW@4      1000e9b0 f   Proclist.obj
 0001:0000d9d0       _ConfigureW@4              1000e9d0 f   Proclist.obj
 0001:0000d9e0       _CompareW@4                1000e9e0 f   Proclist.obj
 0001:0000da00       _OpenW@4                   1000ea00 f   Proclist.obj
 0001:0000dad0       _EncodePointerWrapper@4    1000ead0 f   vc_crt_fix_impl.obj
 0001:0000db20       _DecodePointerWrapper@4    1000eb20 f   vc_crt_fix_impl.obj
 0001:0000db70       _GetModuleHandleExWWrapper@12 1000eb70 f   vc_crt_fix_impl.obj
 0001:0000dbb4       _WNetCancelConnection2W@12 1000ebb4 f   mpr:MPR.dll
 0001:0000dbba       _WNetAddConnection2W@16    1000ebba f   mpr:MPR.dll
 0001:0000dbc0       _VerQueryValueW@16         1000ebc0 f   version:VERSION.dll
 0001:0000dbc6       _GetFileVersionInfoW@16    1000ebc6 f   version:VERSION.dll
 0001:0000dbcc       _GetFileVersionInfoSizeW@8 1000ebcc f   version:VERSION.dll
 0001:0000dbd2       ??_U@YAPAXI@Z              1000ebd2 f   libcpmt:newaop.obj
 0001:0000dbdd       ??_V@YAXPAX@Z              1000ebdd f   LIBCMT:delete2.obj
 0001:0000dbe8       ??0_LocaleUpdate@@QAE@PAUlocaleinfo_struct@@@Z 1000ebe8 f i LIBCMT:memicmp.obj
 0001:0000dc6f       __memicmp_l                1000ec6f f   LIBCMT:memicmp.obj
 0001:0000dd3a       __memicmp                  1000ed3a f   LIBCMT:memicmp.obj
 0001:0000dd8e       _free                      1000ed8e f   LIBCMT:free.obj
 0001:0000ddc8       _malloc                    1000edc8 f   LIBCMT:malloc.obj
 0001:0000de5c       ??3@YAXPAX@Z               1000ee5c f   LIBCMT:delete.obj
 0001:0000de70       _memset                    1000ee70 f   LIBCMT:memset.obj
 0001:0000deea       ??1bad_alloc@std@@UAE@XZ   1000eeea f i LIBCMT:new.obj
 0001:0000def5       ??_Ebad_alloc@std@@UAEPAXI@Z 1000eef5 f i LIBCMT:new.obj
 0001:0000def5       ??_Gbad_alloc@std@@UAEPAXI@Z 1000eef5 f i LIBCMT:new.obj
 0001:0000df1c       ??0bad_alloc@std@@QAE@ABV01@@Z 1000ef1c f i LIBCMT:new.obj
 0001:0000df39       ??2@YAPAXI@Z               1000ef39 f   LIBCMT:new.obj
 0001:0000dfb9       _wcschr                    1000efb9 f   LIBCMT:wcschr.obj
 0001:0000dfe0       _wcspbrk                   1000efe0 f   LIBCMT:wcspbrk.obj
 0001:0000e024       _wcsrchr                   1000f024 f   LIBCMT:wcsrchr.obj
 0001:0000e052       _wcstok                    1000f052 f   LIBCMT:wcstok.obj
 0001:0000e183       __ui64tow                  1000f183 f   LIBCMT:xtow.obj
 0001:0000e1a0       __aulldiv                  1000f1a0 f   LIBCMT:ulldiv.obj
 0001:0000e3ca       _wcstol                    1000f3ca f   LIBCMT:wcstol.obj
 0001:0000e3e4       _wcscspn                   1000f3e4 f   LIBCMT:wcscspn.obj
 0001:0000e430       _memcpy                    1000f430 f   LIBCMT:memcpy.obj
 0001:0000e791       _wcsncat                   1000f791 f   LIBCMT:wcsncat.obj
 0001:0000e7e0       _memmove                   1000f7e0 f   LIBCMT:memmove.obj
 0001:0000eb50       __allmul                   1000fb50 f   LIBCMT:llmul.obj
 0001:0000eb90       __alldiv                   1000fb90 f   LIBCMT:lldiv.obj
 0001:0000ec40       __aullrem                  1000fc40 f   LIBCMT:ullrem.obj
 0001:0000ecb5       __cfltcvt_init             1000fcb5 f   LIBCMT:_fpinit_.obj
 0001:0000ed15       __fpmath                   1000fd15 f   LIBCMT:_fpinit_.obj
 0001:0000ed2e       __CRT_INIT@12              1000fd2e f   LIBCMT:dllcrt0.obj
 0001:0000ef88       __DllMainCRTStartup@12     1000ff88 f   LIBCMT:dllcrt0.obj
 0001:0000f1ce       ___updatetmbcinfo          100101ce f   LIBCMT:mbctype.obj
 0001:0000f2ee       __setmbcp_nolock           100102ee f   LIBCMT:mbctype.obj
 0001:0000f4d7       __setmbcp                  100104d7 f   LIBCMT:mbctype.obj
 0001:0000f671       ___initmbctable            10010671 f   LIBCMT:mbctype.obj
 0001:0000f68f       ___addlocaleref            1001068f f   LIBCMT:localref.obj
 0001:0000f71e       ___removelocaleref         1001071e f   LIBCMT:localref.obj
 0001:0000f7b7       ___freetlocinfo            100107b7 f   LIBCMT:localref.obj
 0001:0000f902       __updatetlocinfoEx_nolock  10010902 f   LIBCMT:localref.obj
 0001:0000f94f       ___updatetlocinfo          1001094f f   LIBCMT:localref.obj
 0001:0000f9c8       __encoded_null             100109c8 f   LIBCMT:tidtable.obj
 0001:0000f9d1       ___crtTlsAlloc@4           100109d1 f   LIBCMT:tidtable.obj
 0001:0000f9da       ___set_flsgetvalue         100109da f   LIBCMT:tidtable.obj
 0001:0000fa0e       __mtterm                   10010a0e f   LIBCMT:tidtable.obj
 0001:0000fa4b       __initptd                  10010a4b f   LIBCMT:tidtable.obj
 0001:0000faff       __getptd_noexit            10010aff f   LIBCMT:tidtable.obj
 0001:0000fb78       __getptd                   10010b78 f   LIBCMT:tidtable.obj
 0001:0000fb92       __freefls@4                10010b92 f   LIBCMT:tidtable.obj
 0001:0000fcc1       __freeptd                  10010cc1 f   LIBCMT:tidtable.obj
 0001:0000fd2f       __mtinit                   10010d2f f   LIBCMT:tidtable.obj
 0001:0000feaa       __tolower_l                10010eaa f   LIBCMT:tolower.obj
 0001:0000ffbf       _tolower                   10010fbf f   LIBCMT:tolower.obj
 0001:0000fff0       ___ascii_memicmp           10010ff0 f   LIBCMT:_memicmp.obj
 0001:00010049       __initp_misc_invarg        10011049 f   LIBCMT:invarg.obj
 0001:00010058       __call_reportfault         10011058 f   LIBCMT:invarg.obj
 0001:00010181       __invoke_watson            10011181 f   LIBCMT:invarg.obj
 0001:000101a6       __invalid_parameter        100111a6 f   LIBCMT:invarg.obj
 0001:000101d3       __invalid_parameter_noinfo 100111d3 f   LIBCMT:invarg.obj
 0001:000101e3       __get_errno_from_oserr     100111e3 f   LIBCMT:dosmap.obj
 0001:00010225       __errno                    10011225 f   LIBCMT:dosmap.obj
 0001:00010238       __heap_init                10011238 f   LIBCMT:heapinit.obj
 0001:00010256       __heap_term                10011256 f   LIBCMT:heapinit.obj
 0001:0001026a       ___crtCorExitProcess       1001126a f   LIBCMT:crt0dat.obj
 0001:00010295       ___crtExitProcess          10011295 f   LIBCMT:crt0dat.obj
 0001:000102ad       __lockexit                 100112ad f   LIBCMT:crt0dat.obj
 0001:000102b6       __unlockexit               100112b6 f   LIBCMT:crt0dat.obj
 0001:000102bf       __init_pointers            100112bf f   LIBCMT:crt0dat.obj
 0001:000102f2       __initterm_e               100112f2 f   LIBCMT:crt0dat.obj
 0001:00010316       __cinit                    10011316 f   LIBCMT:crt0dat.obj
 0001:000104ed       __exit                     100114ed f   LIBCMT:crt0dat.obj
 0001:00010503       __cexit                    10011503 f   LIBCMT:crt0dat.obj
 0001:00010512       __amsg_exit                10011512 f   LIBCMT:crt0dat.obj
 0001:00010530       __GET_RTERRMSG             10011530 f   LIBCMT:crt0msg.obj
 0001:00010556       __NMSG_WRITE               10011556 f   LIBCMT:crt0msg.obj
 0001:00010705       __FF_MSGBANNER             10011705 f   LIBCMT:crt0msg.obj
 0001:0001073e       __initp_heap_handler       1001173e f   LIBCMT:handler.obj
 0001:0001074d       __callnewh                 1001174d f   LIBCMT:handler.obj
 0001:00010775       __VEC_memzero              10011775 f   LIBCMT:p4_memset.obj
 0001:0001082f       ___sse2_available_init     1001182f f   LIBCMT:cpu_disp.obj
 0001:0001083f       ??0exception@std@@QAE@ABQBDH@Z 1001183f f   LIBCMT:stdexcpt.obj
 0001:0001085c       ?what@exception@std@@UBEPBDXZ 1001185c f   LIBCMT:stdexcpt.obj
 0001:00010869       ?_Copy_str@exception@std@@AAEXPBD@Z 10011869 f   LIBCMT:stdexcpt.obj
 0001:000108a9       ?_Tidy@exception@std@@AAEXXZ 100118a9 f   LIBCMT:stdexcpt.obj
 0001:000108c7       ??4exception@std@@QAEAAV01@ABV01@@Z 100118c7 f   LIBCMT:stdexcpt.obj
 0001:000108fc       ??1exception@std@@UAE@XZ   100118fc f   LIBCMT:stdexcpt.obj
 0001:00010907       ??_Eexception@std@@UAEPAXI@Z 10011907 f i LIBCMT:stdexcpt.obj
 0001:00010907       ??_Gexception@std@@UAEPAXI@Z 10011907 f i LIBCMT:stdexcpt.obj
 0001:0001092e       ??0exception@std@@QAE@ABV01@@Z 1001192e f   LIBCMT:stdexcpt.obj
 0001:00010953       ??1type_info@@UAE@XZ       10011953 f   LIBCMT:typinfo.obj
 0001:00010963       ??_Gtype_info@@UAEPAXI@Z   10011963 f i LIBCMT:typinfo.obj
 0001:00010963       ??_Etype_info@@UAEPAXI@Z   10011963 f i LIBCMT:typinfo.obj
 0001:00010a3a       ___onexitinit              10011a3a f   LIBCMT:onexit.obj
 0001:00010a6b       __onexit                   10011a6b f   LIBCMT:onexit.obj
 0001:00010aa7       _atexit                    10011aa7 f   LIBCMT:onexit.obj
 0001:00010abe       __CxxThrowException@8      10011abe f   LIBCMT:throw.obj
 0001:00010b10       __aulldvrm                 10011b10 f   LIBCMT:ulldvrm.obj
 0001:00010ba5       __wchartodigit             10011ba5 f   LIBCMT:wchtodig.obj
 0001:00010d45       _iswctype                  10011d45 f   LIBCMT:iswctype.obj
 0001:00010d9a       __VEC_memcpy               10011d9a f   LIBCMT:p4_memcpy.obj
 0001:00010e9d       __forcdecpt_l              10011e9d f   LIBCMT:cvt.obj
 0001:00010f11       __cropzeros_l              10011f11 f   LIBCMT:cvt.obj
 0001:00010f93       __positive                 10011f93 f   LIBCMT:cvt.obj
 0001:00010faf       __fassign_l                10011faf f   LIBCMT:cvt.obj
 0001:00010ff1       __fassign                  10011ff1 f   LIBCMT:cvt.obj
 0001:0001102a       __forcdecpt                1001202a f   LIBCMT:cvt.obj
 0001:0001103d       __cropzeros                1001203d f   LIBCMT:cvt.obj
 0001:000111b1       __cftoe_l                  100121b1 f   LIBCMT:cvt.obj
 0001:00011278       __cftoe                    10012278 f   LIBCMT:cvt.obj
 0001:00011298       __cftoa_l                  10012298 f   LIBCMT:cvt.obj
 0001:00011711       __cftof_l                  10012711 f   LIBCMT:cvt.obj
 0001:000117d2       __cftog_l                  100127d2 f   LIBCMT:cvt.obj
 0001:000118bf       __cfltcvt_l                100128bf f   LIBCMT:cvt.obj
 0001:00011947       __cfltcvt                  10012947 f   LIBCMT:cvt.obj
 0001:0001196a       __initp_misc_cfltcvt_tab   1001296a f   LIBCMT:cmiscdat.obj
 0001:0001198d       __setdefaultprecision      1001298d f   LIBCMT:fp8.obj
 0001:000119b5       __malloc_crt               100129b5 f   LIBCMT:crtheap.obj
 0001:000119fa       __calloc_crt               100129fa f   LIBCMT:crtheap.obj
 0001:00011a46       __realloc_crt              10012a46 f   LIBCMT:crtheap.obj
 0001:00011a94       __ioinit                   10012a94 f   LIBCMT:ioinit.obj
 0001:00011cd9       __ioterm                   10012cd9 f   LIBCMT:ioinit.obj
 0001:00011d2c       __setenvp                  10012d2c f   LIBCMT:stdenvp.obj
 0001:00011fa2       __setargv                  10012fa2 f   LIBCMT:stdargv.obj
 0001:0001205d       ___crtGetEnvironmentStringsA 1001305d f   LIBCMT:a_env.obj
 0001:000120f4       __RTC_Initialize           100130f4 f   LIBCMT:_initsect_.obj
 0001:0001211a       __RTC_Terminate            1001311a f   LIBCMT:_initsect_.obj
 0001:00012140       __SEH_prolog4              10013140 f   LIBCMT:sehprolg4.obj
 0001:00012185       __SEH_epilog4              10013185 f   LIBCMT:sehprolg4.obj
 0001:000121a0       __except_handler4          100131a0 f   LIBCMT:chandler4.obj
 0001:0001232f       __XcptFilter               1001332f f   LIBCMT:winxfltr.obj
 0001:00012479       ___CppXcptFilter           10013479 f   LIBCMT:winxfltr.obj
 0001:00012499       _DllMain@12                10013499 f   LIBCMT:dllmain.obj
 0001:0001249f       ___security_init_cookie    1001349f f   LIBCMT:gs_support.obj
 0001:0001253a       __freea                    1001353a f i LIBCMT:a_map.obj
 0001:00012741       ___crtLCMapStringA         10013741 f   LIBCMT:a_map.obj
 0001:0001286e       ___crtGetStringTypeA       1001386e f   LIBCMT:a_str.obj
 0001:000128ae       @__security_check_cookie@4 100138ae f   LIBCMT:secchk.obj
 0001:000128bd       __mtinitlocks              100138bd f   LIBCMT:mlock.obj
 0001:00012907       __mtdeletelocks            10013907 f   LIBCMT:mlock.obj
 0001:0001295e       __unlock                   1001395e f   LIBCMT:mlock.obj
 0001:00012975       __mtinitlocknum            10013975 f   LIBCMT:mlock.obj
 0001:00012a37       __lock                     10013a37 f   LIBCMT:mlock.obj
 0001:00012a6a       ___free_lc_time            10013a6a f   LIBCMT:inittime.obj
 0001:00012de1       ___free_lconv_num          10013de1 f   LIBCMT:initnum.obj
 0001:00012e4a       ___free_lconv_mon          10013e4a f   LIBCMT:initmon.obj
 0001:00012f48       __isleadbyte_l             10013f48 f i LIBCMT:_wctype.obj
 0001:00012f80       __isctype_l                10013f80 f   LIBCMT:isctype.obj
 0001:00013038       __crt_debugger_hook        10014038 f   LIBCMT:dbghook.obj
 0001:00013040       _strcspn                   10014040 f   LIBCMT:strcspn.obj
 0001:00013086       _strcpy_s                  10014086 f   LIBCMT:strcpy_s.obj
 0001:000130f0       _strcmp                    100140f0 f   LIBCMT:strcmp.obj
 0001:00013180       _strlen                    10014180 f   LIBCMT:strlen.obj
 0001:00013210       _strpbrk                   10014210 f   LIBCMT:strpbrk.obj
 0001:00013250       ?terminate@@YAXXZ          10014250 f   LIBCMT:hooks.obj
 0001:00013289       __initp_eh_hooks           10014289 f   LIBCMT:hooks.obj
 0001:0001329a       __initp_misc_winsig        1001429a f   LIBCMT:winsig.obj
 0001:000132ef       ___get_sigabrt             100142ef f   LIBCMT:winsig.obj
 0001:000132fc       _raise                     100142fc f   LIBCMT:winsig.obj
 0001:0001349f       __initp_misc_rand_s        1001449f f   LIBCMT:rand_s.obj
 0001:000134ae       __initp_misc_purevirt      100144ae f   LIBCMT:inithelp.obj
 0001:000134c0       __ValidateImageBase        100144c0 f   LIBCMT:pesect.obj
 0001:00013500       __FindPESection            10014500 f   LIBCMT:pesect.obj
 0001:00013550       __IsNonwritableInCurrentImage 10014550 f   LIBCMT:pesect.obj
 0001:0001360c       ___crtMessageBoxW          1001460c f   LIBCMT:crtmboxw.obj
 0001:00013778       _wcscat_s                  10014778 f   LIBCMT:wcscat_s.obj
 0001:000137ed       _wcsncpy_s                 100147ed f   LIBCMT:wcsncpy_s.obj
 0001:000138ba       _wcslen                    100148ba f   LIBCMT:wcslen.obj
 0001:000138d5       _wcscpy_s                  100148d5 f   LIBCMT:wcscpy_s.obj
 0001:00013938       __set_error_mode           10014938 f   LIBCMT:errmode.obj
 0001:00013977       ?_Type_info_dtor@type_info@@CAXPAV1@@Z 10014977 f   LIBCMT:typname.obj
 0001:000139e7       __msize                    100149e7 f   LIBCMT:msize.obj
 0001:00013a20       _strrchr                   10014a20 f   LIBCMT:strrchr.obj
 0001:00013a4d       __isdigit_l                10014a4d f i LIBCMT:_ctype.obj
 0001:00013a9e       _isdigit                   10014a9e f i LIBCMT:_ctype.obj
 0001:00013acc       __atodbl_l                 10014acc f   LIBCMT:atodbl.obj
 0001:00013b74       __atoflt_l                 10014b74 f   LIBCMT:atodbl.obj
 0001:00013c1c       __fptostr                  10014c1c f   LIBCMT:_fptostr.obj
 0001:00013ccf       ___dtold                   10014ccf f   LIBCMT:_cfout_.obj
 0001:00013d82       __fltout2                  10014d82 f   LIBCMT:_cfout_.obj
 0001:00013e10       __alldvrm                  10014e10 f   LIBCMT:lldvrm.obj
 0001:00013ef0       __aullshr                  10014ef0 f   LIBCMT:ullshr.obj
 0001:00013f0f       __fptrap                   10014f0f f   LIBCMT:crt0fp.obj
 0001:00013f18       __controlfp_s              10014f18 f   LIBCMT:_contrlfp_.obj
 0001:00013f77       __calloc_impl              10014f77 f   LIBCMT:calloc_impl.obj
 0001:00013ff9       _realloc                   10014ff9 f   LIBCMT:realloc.obj
 0001:000140f9       __ismbblead                100150f9 f   LIBCMT:ismbbyte.obj
 0001:00014120       __local_unwind4            10015120 f   LIBCMT:exsup4.obj
 0001:000141f6       __seh_longjmp_unwind4@4    100151f6 f   LIBCMT:exsup4.obj
 0001:00014212       @_EH4_CallFilterFunc@8     10015212 f   LIBCMT:exsup4.obj
 0001:00014229       @_EH4_TransferToHandler@8  10015229 f   LIBCMT:exsup4.obj
 0001:00014242       @_EH4_GlobalUnwind2@8      10015242 f   LIBCMT:exsup4.obj
 0001:0001425b       @_EH4_LocalUnwind@16       1001525b f   LIBCMT:exsup4.obj
 0001:00014280       __alloca_probe_16          10015280 f   LIBCMT:alloca16.obj
 0001:00014296       __alloca_probe_8           10015296     LIBCMT:alloca16.obj
 0001:000142ac       ___report_gsfailure        100152ac f   LIBCMT:gs_report.obj
 0001:000143b2       _abort                     100153b2 f   LIBCMT:abort.obj
 0001:000143e5       __ld12tod                  100153e5 f   LIBCMT:_intrncvt_.obj
 0001:00014936       __ld12tof                  10015936 f   LIBCMT:_intrncvt_.obj
 0001:00014e87       ___strgtold12_l            10015e87 f   LIBCMT:_strgtold_.obj
 0001:00015563       _$I10_OUTPUT               10016563 f   LIBCMT:_x10fout_.obj
 0001:00015f89       __control87                10016f89 f i LIBCMT:_ieee87_.obj
 0001:000162a0       __global_unwind2           100172a0 f   LIBCMT:exsup.obj
 0001:00016305       __local_unwind2            10017305 f   LIBCMT:exsup.obj
 0001:00016389       __abnormal_termination     10017389 f   LIBCMT:exsup.obj
 0001:000163ac       __NLG_Notify1              100173ac f   LIBCMT:exsup.obj
 0001:000163b5       __NLG_Notify               100173b5 f   LIBCMT:exsup.obj
 0001:000163cc       __NLG_Dispatch             100173cc     LIBCMT:exsup.obj
 0001:000163cc       __NLG_Dispatch2            100173cc     LIBCMT:exsup.obj
 0001:000163d4       __NLG_Call                 100173d4 f   LIBCMT:exsup.obj
 0001:000163d6       __NLG_Return2              100173d6     LIBCMT:exsup.obj
 0001:000163e0       ___ascii_strnicmp          100173e0 f   LIBCMT:_strnicm.obj
 0001:00016441       ___mtold12                 10017441 f   LIBCMT:_mantold_.obj
 0001:00016625       ___set_fpsr_sse2           10017625 f   LIBCMT:_fpctrl_.obj
 0001:00016698       _RtlUnwind@16              10017698 f   kernel32:KERNEL32.dll
 0001:0001669e       __wcsdup                   1001769e f   LIBCMT:wcsdup.obj
 0001:0001669e       _wcsdup                    1001769e f   LIBCMT:wcsdup.obj
 0001:000166f3       _calloc                    100176f3 f   LIBCMT:calloc.obj
 0001:00016748       __TI2?AVbad_alloc@std@@    10017748     LIBCMT:new.obj
 0001:00016758       __CTA2?AVbad_alloc@std@@   10017758     LIBCMT:new.obj
 0001:00016764       __CT??_R0?AVbad_alloc@std@@@8??0bad_alloc@std@@QAE@ABV01@@Z12 10017764     LIBCMT:new.obj
 0001:00016780       __CT??_R0?AVexception@std@@@8??0exception@std@@QAE@ABV01@@Z12 10017780     LIBCMT:new.obj
 0001:0001698c       __IMPORT_DESCRIPTOR_KERNEL32 1001798c     kernel32:KERNEL32.dll
 0001:000169a0       __IMPORT_DESCRIPTOR_USER32 100179a0     user32:USER32.dll
 0001:000169b4       __IMPORT_DESCRIPTOR_ADVAPI32 100179b4     advapi32:ADVAPI32.dll
 0001:000169c8       __IMPORT_DESCRIPTOR_ole32  100179c8     ole32:ole32.dll
 0001:000169dc       __IMPORT_DESCRIPTOR_MPR    100179dc     mpr:MPR.dll
 0001:000169f0       __IMPORT_DESCRIPTOR_VERSION 100179f0     version:VERSION.dll
 0001:00016a04       __IMPORT_DESCRIPTOR_OLEAUT32 10017a04     oleaut32:OLEAUT32.dll
 0001:00016a18       __NULL_IMPORT_DESCRIPTOR   10017a18     kernel32:KERNEL32.dll
 0002:00000000       ?DescIDs@@3PAHA            10019000     Pclass.obj
 0002:00000080       ?Counters@@3PAU_Counters@@A 10019080     perfthread.obj
 0002:00000188       ?pNtQueryInformationProcess@@3P6GJPAXW4_PROCESSINFOCLASS@@0KPAK@ZA 10019188     Proclist.obj
 0002:0000018c       ?pNtQueryInformationThread@@3P6GJPAXK0KPAK@ZA 1001918c     Proclist.obj
 0002:00000190       ?pNtQueryObject@@3P6GJPAXK0K0@ZA 10019190     Proclist.obj
 0002:00000194       ?pNtQuerySystemInformation@@3P6GJKPAXKPAK@ZA 10019194     Proclist.obj
 0002:00000198       ?pNtQueryInformationFile@@3P6GJPAX00KK@ZA 10019198     Proclist.obj
 0002:0000019c       ?pIsWow64Process@@3P6GHPAXPAH@ZA 1001919c     Proclist.obj
 0002:000001a0       ?pGetGuiResources@@3P6GKPAXK@ZA 100191a0     Proclist.obj
 0002:000001a4       ?pIsValidSid@@3P6GHPAX@ZA  100191a4     Proclist.obj
 0002:000001a8       ?pGetSidIdentifierAuthority@@3P6GPAU_SID_IDENTIFIER_AUTHORITY@@PAX@ZA 100191a8     Proclist.obj
 0002:000001ac       ?pGetSidSubAuthorityCount@@3P6GPAEPAX@ZA 100191ac     Proclist.obj
 0002:000001b0       ?pGetSidSubAuthority@@3P6GPAKPAXK@ZA 100191b0     Proclist.obj
 0002:000001b4       ?pLookupAccountName@@3P6GHPB_W0PAXPAKPA_W2PAW4_SID_NAME_USE@@@ZA 100191b4     Proclist.obj
 0002:000001b8       ?pCoSetProxyBlanket@@3P6GJPAUIUnknown@@KKPA_WKKPAXK@ZA 100191b8     Proclist.obj
 0002:000001c0       ??_R0?AVbad_alloc@std@@@8  100191c0     LIBCMT:new.obj
 0002:000001dc       ??_R0?AVexception@std@@@8  100191dc     LIBCMT:new.obj
 0002:00000200       __fltused                  10019200     LIBCMT:_fpinit_.obj
 0002:00000204       __ldused                   10019204     LIBCMT:_fpinit_.obj
 0002:00000208       ___initialmbcinfo          10019208     LIBCMT:mbctype.obj
 0002:00000428       __mbctype                  10019428     LIBCMT:mbctype.obj
 0002:00000530       __mbcasemap                10019530     LIBCMT:mbctype.obj
 0002:00000630       ___ptmbcinfo               10019630     LIBCMT:mbctype.obj
 0002:00000728       ___globallocalestatus      10019728     LIBCMT:glstatus.obj
 0002:0000072c       ___clocalestr              1001972c     LIBCMT:nlsdata2.obj
 0002:00000730       ___lc_time_c               10019730     LIBCMT:nlsdata2.obj
 0002:00000898       ___initiallocinfo          10019898     LIBCMT:nlsdata2.obj
 0002:00000970       ___ptlocinfo               10019970     LIBCMT:nlsdata2.obj
 0002:00000974       ___flsindex                10019974     LIBCMT:tidtable.obj
 0002:00000978       ___getvalueindex           10019978     LIBCMT:tidtable.obj
 0002:00000af4       ??_R0?AVtype_info@@@8      10019af4     LIBCMT:typinfo.obj
 0002:00000b10       __cfltcvt_tab              10019b10     LIBCMT:cmiscdat.obj
 0002:00000b38       ___badioinfo               10019b38     LIBCMT:ioinit.obj
 0002:00000b80       ___security_cookie         10019b80     LIBCMT:gs_cookie.obj
 0002:00000b84       ___security_cookie_complement 10019b84     LIBCMT:gs_cookie.obj
 0002:00000ca8       ___lconv_static_decimal    10019ca8     LIBCMT:lconv.obj
 0002:00000cac       ___lconv_static_W_decimal  10019cac     LIBCMT:lconv.obj
 0002:00000cb0       ___lconv_c                 10019cb0     LIBCMT:lconv.obj
 0002:00000d00       ___lconv                   10019d00     LIBCMT:lconv.obj
 0002:00000d04       __pctype                   10019d04     LIBCMT:ctype.obj
 0002:00000d08       __pwctype                  10019d08     LIBCMT:ctype.obj
 0002:00000d0c       ___mb_cur_max              10019d0c     LIBCMT:nlsdata1.obj
 0002:00000d10       ___decimal_point           10019d10     LIBCMT:nlsdata1.obj
 0002:00000d14       ___decimal_point_length    10019d14     LIBCMT:nlsdata1.obj
 0002:00000d20       ___abort_behavior          10019d20     LIBCMT:abort.obj
 0002:00000d60       __NLG_Destination          10019d60     LIBCMT:exsup.obj
 0002:00000d70       __pow10pos                 10019d70     LIBCMT:_constpow_.obj
 0002:00000ed0       __pow10neg                 10019ed0     LIBCMT:_constpow_.obj
 0002:00001060       ?FPRINTFbuffer@@3PA_WA     1001a060     fileio.obj
 0002:00021268       ?ProcPanelModesRemote@Plist@@2PAY0FA@_WA 1003a268     Pclass.obj
 0002:000218a8       ?PanelModesRemote@Plist@@2PAUPanelMode@@A 1003a8a8     Pclass.obj
 0002:000219e8       ?bInit@Plist@@2_NA         1003a9e8     Pclass.obj
 0002:000219f0       ?PanelModesLocal@Plist@@2PAUPanelMode@@A 1003a9f0     Pclass.obj
 0002:00021b30       ?ProcPanelModesLocal@Plist@@2PAY0FA@_WA 1003ab30     Pclass.obj
 0002:00022170       ?PanelModeBuffer@Plist@@2PA_WA 1003b170     Pclass.obj
 0002:00025e70       ?hDebugToken@DebugToken@@0RAXA 1003ee70     Plist.obj
 0002:00025ec8       ?Info@@3UPluginStartupInfo@@A 1003eec8     Proclist.obj
 0002:00025f50       ?_ui64Table@@3PAVui64Table@@A 1003ef50     Proclist.obj
 0002:00025f54       ?PluginRootKey@@3PA_WA     1003ef54     Proclist.obj
 0002:00025f58       ?FSF@@3UFarStandardFunctions@@A 1003ef58     Proclist.obj
 0002:00026014       ?Opt@@3U_Opt@@A            1003f014     Proclist.obj
 0002:00026070       ___fastflag                1003f070     LIBCMT:_fpinit_.obj
 0002:00026078       __aenvptr                  1003f078     LIBCMT:dllcrt0.obj
 0002:0002607c       __wenvptr                  1003f07c     LIBCMT:dllcrt0.obj
 0002:00026080       ___error_mode              1003f080     LIBCMT:dllcrt0.obj
 0002:00026084       ___app_type                1003f084     LIBCMT:dllcrt0.obj
 0002:0002608c       ___mbulinfo                1003f08c     LIBCMT:mbctype.obj
 0002:00026098       ___mbcodepage              1003f098     LIBCMT:mbctype.obj
 0002:0002609c       ___ismbcodepage            1003f09c     LIBCMT:mbctype.obj
 0002:000260a0       ___mblcid                  1003f0a0     LIBCMT:mbctype.obj
 0002:000260a4       _gpFlsAlloc                1003f0a4     LIBCMT:tidtable.obj
 0002:000260a8       _gpFlsGetValue             1003f0a8     LIBCMT:tidtable.obj
 0002:000260ac       _gpFlsSetValue             1003f0ac     LIBCMT:tidtable.obj
 0002:000260b0       _gpFlsFree                 1003f0b0     LIBCMT:tidtable.obj
 0002:000260b4       ___pInvalidArgHandler      1003f0b4     LIBCMT:invarg.obj
 0002:000260b8       ___locale_changed          1003f0b8     LIBCMT:setlocal.obj
 0002:000260bc       __crtheap                  1003f0bc     LIBCMT:heapinit.obj
 0002:000260c0       __umaskval                 1003f0c0     LIBCMT:crt0dat.obj
 0002:000260c4       ___argc                    1003f0c4     LIBCMT:crt0dat.obj
 0002:000260c8       ___argv                    1003f0c8     LIBCMT:crt0dat.obj
 0002:000260cc       ___wargv                   1003f0cc     LIBCMT:crt0dat.obj
 0002:000260d0       __environ                  1003f0d0     LIBCMT:crt0dat.obj
 0002:000260d4       ___initenv                 1003f0d4     LIBCMT:crt0dat.obj
 0002:000260d8       __wenviron                 1003f0d8     LIBCMT:crt0dat.obj
 0002:000260dc       ___winitenv                1003f0dc     LIBCMT:crt0dat.obj
 0002:000260e0       __pgmptr                   1003f0e0     LIBCMT:crt0dat.obj
 0002:000260e4       __wpgmptr                  1003f0e4     LIBCMT:crt0dat.obj
 0002:000260e8       __exitflag                 1003f0e8     LIBCMT:crt0dat.obj
 0002:000260ec       __C_Termination_Done       1003f0ec     LIBCMT:crt0dat.obj
 0002:000260f0       __C_Exit_Done              1003f0f0     LIBCMT:crt0dat.obj
 0002:00026720       ?_pnhHeap@@3P6AHI@ZA       1003f720     LIBCMT:handler.obj
 0002:00026724       __newmode                  1003f724     LIBCMT:_newmode.obj
 0002:00026728       __maxwait                  1003f728     LIBCMT:crtheap.obj
 0002:00026988       ___lconv_static_null       1003f988     LIBCMT:lconv.obj
 0002:0002698c       ___lconv_static_W_null     1003f98c     LIBCMT:lconv.obj
 0002:00026990       ?__pInconsistency@@3P6AXXZA 1003f990     LIBCMT:hooks.obj
 0002:000269ac       ___pPurecall               1003f9ac     LIBCMT:inithelp.obj
 0002:000269cc       __outputformat             1003f9cc     LIBCMT:outputformat.obj
 0002:00026d08       ?pArgList@UnDecorator@@0PAVReplicator@@A 1003fd08     LIBCMT:undname.obj
 0002:00026d0c       ?pZNameList@UnDecorator@@0PAVReplicator@@A 1003fd0c     LIBCMT:undname.obj
 0002:00026d10       ?pTemplateArgList@UnDecorator@@0PAVReplicator@@A 1003fd10     LIBCMT:undname.obj
 0002:00026d14       ?gName@UnDecorator@@0PBDB  1003fd14     LIBCMT:undname.obj
 0002:00026d18       ?name@UnDecorator@@0PBDB   1003fd18     LIBCMT:undname.obj
 0002:00026d1c       ?outputString@UnDecorator@@0PADA 1003fd1c     LIBCMT:undname.obj
 0002:00026d20       ?maxStringLength@UnDecorator@@0HA 1003fd20     LIBCMT:undname.obj
 0002:00026d24       ?disableFlags@UnDecorator@@0KA 1003fd24     LIBCMT:undname.obj
 0002:00026d28       ?m_pGetParameter@UnDecorator@@0P6APADJ@ZA 1003fd28     LIBCMT:undname.obj
 0002:00026d2c       ?fExplicitTemplateParams@UnDecorator@@0_NA 1003fd2c     LIBCMT:undname.obj
 0002:00026d2d       ?fGetTemplateArgumentList@UnDecorator@@0_NA 1003fd2d     LIBCMT:undname.obj
 0002:00026d30       __debugger_hook_dummy      1003fd30     <common>
 0002:00026d34       __pDestructExceptionObject 1003fd34     <common>
 0002:00026d38       __nhandle                  1003fd38     <common>
 0002:00026d40       ___pioinfo                 1003fd40     <common>
 0002:00026e40       ___sse2_available          1003fe40     <common>
 0002:00026e44       ___env_initialized         1003fe44     <common>
 0002:00026e48       ___onexitend               1003fe48     <common>
 0002:00026e4c       ___onexitbegin             1003fe4c     <common>
 0002:00026e50       ___mbctype_initialized     1003fe50     <common>
 0002:00026e54       ___dyn_tls_init_callback   1003fe54     <common>
 0002:00026e58       __acmdln                   1003fe58     <common>

 entry point at        0001:0000ef88

 Static symbols

 0001:00003ec0       ?GetProcessId@@YAHPAXAAK@Z 10004ec0 f   handles.obj
 0001:00003f10       ?GetFileNameThread@@YGKPAX@Z 10004f10 f   handles.obj
 0001:00003f50       ?PrintFileName@@YA_NPAX0@Z 10004f50 f   handles.obj
 0001:00004050       ?GetTypeToken@@YA_NPAXPA_WK@Z 10005050 f   handles.obj
 0001:000040d0       ?GetTypeFromTypeToken@@YAGPB_W@Z 100050d0 f   handles.obj
 0001:00004110       ?PrintNameByType@@YA_NPAXG0PAVPerfThread@@@Z 10005110 f   handles.obj
 0001:00004410       ?PrintNameAndType@@YA_NPAXK0PAVPerfThread@@@Z 10005410 f   handles.obj
 0001:00004570       ?ConvertSid@@YAHPAXPA_WPAK@Z 10005570 f   handles.obj
 0001:000046a0       ?GetUserAccountID@@YAPB_WXZ 100056a0 f   handles.obj
 0001:00004ef0       ?fIsValidSid@@YGHPAX@Z     10005ef0 f i PCFG.OBJ
 0001:00004ef0       ?fGetSidIdentifierAuthority@@YGPAU_SID_IDENTIFIER_AUTHORITY@@PAX@Z 10005ef0 f i PCFG.OBJ
 0001:00004ef0       ?fGetSidSubAuthorityCount@@YGPAEPAX@Z 10005ef0 f i PCFG.OBJ
 0001:00004f10       ?fGetSidSubAuthority@@YGPAKPAXK@Z 10005f10 f i PCFG.OBJ
 0001:00004f10       ?fIsWow64Process@@YGHPAXPAH@Z 10005f10 f i PCFG.OBJ
 0001:00004f10       ?fGetGuiResources@@YGKPAXK@Z 10005f10 f i PCFG.OBJ
 0001:00005f10       ?ui64toa_width@@YAX_KPA_WI_N@Z 10006f10 f   Pclass.obj
 0001:00006690       ?GenerateTitles@@YAXQAY0FA@_WPAUPanelMode@@QAY0BI@PA_W@Z 10007690 f   Pclass.obj
 0001:0000a960       ?getcounter@@YAHPA_W@Z     1000b960 f   perfthread.obj
 0001:0000ba40       ?FreeUserData@@YGXPAXPBUFarPanelItemFreeInfo@@@Z 1000ca40 f   Plist.obj
 0001:0000d540       ?fNtQuerySystemInformation@@YGJKPAXKPAK@Z 1000e540 f   Proclist.obj
 0001:0000d550       ?fNtQueryInformationProcess@@YGJPAXW4_PROCESSINFOCLASS@@0KPAK@Z 1000e550 f   Proclist.obj
 0001:0000d550       ?fNtQueryInformationFile@@YGJPAX00KK@Z 1000e550 f   Proclist.obj
 0001:0000d550       ?fNtQueryObject@@YGJPAXK0K0@Z 1000e550 f   Proclist.obj
 0001:0000d550       ?fNtQueryInformationThread@@YGJPAXK0KPAK@Z 1000e550 f   Proclist.obj
 0001:0000d560       ?fLookupAccountName@@YGHPB_W0PAXPAKPA_W2PAW4_SID_NAME_USE@@@Z 1000e560 f   Proclist.obj
 0001:0000d570       ?fCoSetProxyBlanket@@YGJPAUIUnknown@@KKPA_WKKPAXK@Z 1000e570 f   Proclist.obj
 0001:0000d580       ?dynamic_bind@@YAXXZ       1000e580 f   Proclist.obj
 0001:0000da80       ?DecodePointer@implementation@?1??DecodePointerWrapper@@9@4@SGPAXPAX@Z 1000ea80 f   vc_crt_fix_impl.obj
 0001:0000da80       ?EncodePointer@implementation@?1??EncodePointerWrapper@@9@4@SGPAXPAX@Z 1000ea80 f   vc_crt_fix_impl.obj
 0001:0000da90       ?GetModuleHandleExW@implementation@?1??GetModuleHandleExWWrapper@@9@12@SGHKPB_WPAPAUHINSTANCE__@@@Z 1000ea90 f   vc_crt_fix_impl.obj
 0001:0000e100       @x64tow@20                 1000f100 f   LIBCMT:xtow.obj
 0001:0000e208       ?wcstoxl@@YAKPB_WPAPB_WHH@Z 1000f208 f   LIBCMT:wcstol.obj
 0001:0000ee92       ___DllMainCRTStartup       1000fe92 f   LIBCMT:dllcrt0.obj
 0001:0000efab       ?CPtoLCID@@YAHH@Z          1000ffab f   LIBCMT:mbctype.obj
 0001:0000efda       ?setSBCS@@YAXPAUthreadmbcinfostruct@@@Z 1000ffda f   LIBCMT:mbctype.obj
 0001:0000f03e       ?setSBUpLow@@YAXPAUthreadmbcinfostruct@@@Z 1001003e f   LIBCMT:mbctype.obj
 0001:0000f272       ?getSystemCP@@YAHH@Z       10010272 f   LIBCMT:mbctype.obj
 0001:000103ad       _doexit                    100113ad f   LIBCMT:crt0dat.obj
 0001:00010984       __onexit_nolock            10011984 f   LIBCMT:onexit.obj
 0001:0001100b       __shift                    1001200b f   LIBCMT:cvt.obj
 0001:00011050       __cftoe2_l                 10012050 f   LIBCMT:cvt.obj
 0001:0001160e       __cftof2_l                 1001260e f   LIBCMT:cvt.obj
 0001:00011e08       _parse_cmdline             10012e08 f   LIBCMT:stdargv.obj
 0001:0001255a       ?__crtLCMapStringA_stat@@YAHPAUlocaleinfo_struct@@KKPBDHPADHHH@Z 1001355a f   LIBCMT:a_map.obj
 0001:00012787       ?__crtGetStringTypeA_stat@@YAHPAUlocaleinfo_struct@@KPBDHPAGHHH@Z 10013787 f   LIBCMT:a_str.obj
 0001:000132b8       _siglookup                 100142b8 f   LIBCMT:winsig.obj
 0001:000140a6       ?x_ismbbtype_l@@YAHPAUlocaleinfo_struct@@IHH@Z 100150a6 f   LIBCMT:ismbbyte.obj
 0001:000141b0       __unwind_handler4          100151b0 f   LIBCMT:exsup4.obj
 0001:00015e5b       __hw_cw                    10016e5b f   LIBCMT:_ieee87_.obj
 0001:00015ee9       ___hw_cw_sse2              10016ee9 f   LIBCMT:_ieee87_.obj
 0001:000162c0       __unwind_handler           100172c0 f   LIBCMT:exsup.obj
 0001:00016733       ??__Fnomem@?5???2@YAPAXI@Z@YAXXZ 10017733 f   LIBCMT:new.obj
